:100000000C941E060C94E9280C9416290C944606B0
:100010000C9446060C9446060C9446060C94460630
:100020000C9446060C9446060C9422130C94460637
:100030000C9446060C9446060C9446060C94460610
:100040000C9443290C9446060C94312D0C94742D79
:100050000C9446060C9446060C9446060C944606F0
:100060000C9446060C9446062A198C196B196E19C5
:100070007119741977197A197D198C198619BE1A94
:10008000C01AC01ABE1AC01AC01AC01AC01AC01AA2
:10009000C01AC01AC01AC01AC01AC01AC01AC01A90
:1000A000441AC01AC01AC01AC01AC01AB519C01A08
:1000B000C01AC01AC01AC01AC01AC01AC01AC01A70
:1000C000C01AC01AC01AC01AC01AC01A501A501A40
:1000D000501A501A501A501A501A501A501AC01A60
:1000E000C01AC01AC01AC01AC01AB5194F1A4F1A2E
:1000F0004F1A4F1AC01A5D1A631A691A6F1A751AC5
:100100007B1A811A871A911A9B1AA51AAF1AF61927
:10011000B819C01AC01AC01AC01A441AC01AC01A94
:10012000C01AC01AC01AC01AC01AC01A4E1A4E1AE3
:100130004E1A4E1AC01A5D1A631A691A6F1A751A86
:100140007B1A811A871A911A9B1AA51AAF1AF619E7
:10015000B819C01AC01AC01AC01A441AF31AF31AEE
:10016000F31AF31AF31AF31AF31AF31AF31AF31A27
:10017000F31AF31AF31A091C091C091C091C091C9F
:10018000091C381B421B4C1B561BB31BBD1BCC1B35
:10019000DD1B651D7A1D861D8F1D9E1DC31DCC1D7B
:1001A000151EDE1D2A21302136213D214B216D21D6
:1001B0008B21456E746572206D656E752E2E2E0036
:1001C000546F67676C6564206D6963726F50504D42
:1001D00000546F67676C656420696E76657274653C
:1001E000642050504D2100546F67676C6564205443
:1001F00058206D7574696E672100546F67676C6570
:10020000642074656C656D65747279210050726F3D
:10021000746F636F6C206572726F72207769746897
:100220002052580054696D656F7574207768656E4B
:1002300020636F6E6E656374696E6720746F205201
:100240005800507265737320616E79206B65792058
:10025000746F2063616E63656C00436F6E6E6563DF
:1002600074696E6720746F2052582C20706F776508
:100270007220757020746865205258202877697440
:10028000682062696E6420706C7567206966206EF4
:100290006F74207573696E6720616C776179732064
:1002A00062696E642900546F67676C656420276912
:1002B0006D6D656469617465206F75747075742700
:1002C00000546F67676C65642027736C61766520E6
:1002D0006D6F64652700546F67676C6564202761E4
:1002E0006C776179732062696E642700546F676769
:1002F0006C65642050504D206368616E6E656C20A3
:100300006C696D69740053657420525353492069B8
:100310006E6A656374696F6E206368616E6E656C8A
:100320002028303D3D64697361626C652900536526
:10033000742050504D206D696E696D756D20737914
:100340006E630053657420626561636F6E20696E31
:1003500074657276616C0053657420626561636FC9
:100360006E2064656C617900536574206265616319
:100370006F6E206672657175656E637920696E2097
:10038000487A3A20303D64697361626C652C205074
:10039000783D504D52206368616E6E656C20782CFC
:1003A0002046783D465253206368616E6E656C202E
:1003B00078005365742050574D2073746F7020641B
:1003C000656C61792028302064697361626C6564B2
:1003D0002C20312D323535203D3D20302E317320FB
:1003E0002D2035306D696E29005365742050504DB5
:1003F0002073746F702064656C61792028302064EC
:10040000697361626C65642C20312D323535203D75
:100410003D20302E3173202D2035306D696E29003E
:10042000536574206661696C736166652064656CF0
:1004300061792028302064697361626C65642C20C6
:10044000312D323535203D3D20302E3173202D2089
:1004500035306D696E29002A2A2A2A2A2A2A2A2A50
:100460002A2A2A2A2A2A2A2A2A2A2A2A2A2A2A2AEC
:100470002A2A2A2A0052582041636B6564202D20C5
:1004800072657665727420737563636573736675E0
:100490006C21002A2A2A2A2A2A2A2A2A2A2A2A2AAD
:1004A0002A2A2A2A2A2A2A2A2A2A2A2A2A2A2A2AAC
:1004B000002A2A2A2A2A2A2A2A2A2A2A2A2A2A2AC6
:1004C0002A2A2A2A2A2A2A2A2A2A2A2A2A2A00528E
:1004D000582041636B6564202D20757064617465DC
:1004E000207375636365737366756C21002A2A2A0D
:1004F0002A2A2A2A2A2A2A2A2A2A2A2A2A2A2A2A5C
:100500002A2A2A2A2A2A2A2A2A2A0056616C696457
:100510002063686F69636573206172653A205B319F
:100520005D2D5B31365D20286368616E6E656C20E1
:10053000312D31362900536574206F7574707574D0
:1005400020666F7220706F727420005B585D2061AE
:10055000626F7274206368616E67657320616E6498
:10056000206578697420525820636F6E6669670051
:100570005B535D20736176652073657474696E6783
:100580007320746F205258005B525D20726576654F
:1005900072742052582073657474696E6773207486
:1005A0006F2064656661756C747300557365206EA9
:1005B000756D62657273205B312D445D20746F2010
:1005C0006564697420706F727473205B452D515D92
:1005D00020666F722073657474696E677300202DD6
:1005E00020726563656976657220636F6E66696700
:1005F000757261746F722C20727820737720000AF4
:100600000A6F70656E4C52536E67200053657420FC
:1006100073657269616C2062617564726174653AB8
:10062000200056616C69642063686F696365733A82
:100630002031202D20342B34202F2032202D203823
:10064000202F2033202D20382B34202F2034202D14
:10065000203132202F2035202D2031322B34202FF5
:100660002036202D20313600536574204368616E9A
:100670006E656C20636F6E6669673A20005365741F
:100680002044617461726174652028302D32293AEA
:10069000200053657420486F70206368616E6E653A
:1006A0006C7320286D61782032342C207365706162
:1006B000726174656420627920636F6D6D61732966
:1006C0002076616C69642076616C75657320312DCC
:1006D0003235353A2000536574206368616E6E656B
:1006E0006C2073706163696E6720287831306B48C5
:1006F0007A293A200053657420524620706F77653E
:10070000722028302D37293A200053657420524634
:10071000206D6167696320286865782920652E67E8
:100720002E20307844454144463030443A2000532E
:1007300065742062617365206672657175656E63AC
:10074000792028696E20487A293A20005B5A5D207A
:10075000656E746572207265636569766572206383
:100760006F6E66696775726174696F6E2075746902
:100770006C79005B465D20646973706C61792061FF
:10078000637475616C206672657175656E63696509
:10079000732075736564005B525D2063616C6375E3
:1007A0006C6174652072616E646F6D206B65792079
:1007B000616E6420686F70206C697374005B495DC2
:1007C000207265696E697469616C697A6520736508
:1007D0007474696E677320746F20736B65746368DB
:1007E0002064656661756C7473005B585D2072658A
:1007F00076657274206368616E67657320616E64EC
:100800002065786974206D656E75005B535D20739B
:100810006176652073657474696E677320746F20E8
:10082000454550524F4D20616E64206578697420B3
:100830006D656E7500557365206E756D62657273BA
:10084000205B302D395D20746F20656469742070E1
:100850006172616D657465727300202D2053797328
:1008600074656D20636F6E66696775726174696F18
:100870006E000A0A6F70656E4C52536E672000510D
:1008800029204F7574707574206265666F726520DB
:100890006C696E6B20283D465329203A2000502970
:1008A00020536C617665206D6F64652028657870D3
:1008B0006572696D656E74616C293A20004F29205C
:1008C00054696D65642042494E44206174207374FC
:1008D000617274757020203A20004E292050504DCE
:1008E000206F7574707574206C696D69746564200F
:1008F000202020203A200044495341424C454400E6
:100900004D292050504D205253534920746F20637D
:1009100068616E6E656C202020203A20004C2920F2
:1009200050504D206D696E696D756D2073796E63E1
:10093000202875732920203A200044495341424C15
:100940004544004B29204661696C736166652062ED
:100950006561636F6E20696E74762E2028312D32AA
:10096000353573293A20004A29204661696C736144
:10097000666520626561636F6E2064656C617920D5
:1009800028302D323535203D3E20313073202D204A
:100990003135306D696E293A200049292046616958
:1009A0006C7361666520626561636F6E206672714B
:1009B0002E203A200048292050574D2073746F7024
:1009C0002064656C6179202020202020203A2000BE
:1009D00047292050504D2073746F702064656C61FE
:1009E00079202020202020203A200046292046611E
:1009F000696C736166652064656C617920202020D4
:100A00002020203A200050574D206368616E6E65AB
:100A10006C200066756E6374696F6E3A2000292041
:100A2000706F72742000506F776572546F776572C3
:100A300000445446205548462033322D62697420C4
:100A400031306368004F70656E4C52536E67525878
:100A5000206D696E6920342F36636800466C7974A6
:100A6000726F6E2F4F72616E6765525820554846FF
:100A70002038636800525820747970653A20004429
:100A8000697361626C656400487A00203D3D200016
:100A900043616C63756C61746564207061636B6540
:100AA0007420696E74657276616C3A200042292068
:100AB0004D6963726F202868616C66292050504D23
:100AC000202020203A00412920496E766572746505
:100AD000642050504D20696E20202020203A0030A4
:100AE00029204D7574652062757A7A657220286DAB
:100AF0006F73746C79293A003929205365726961E2
:100B00006C2062617564726174653A00736D617224
:100B100074506F7274004672536B79005472616E38
:100B200073706172656E740044697361626C6564B0
:100B30000038292054656C656D657472793A2020FF
:100B40002020202020003729204368616E6E656CCC
:100B500020636F6E6669673A202000362920446161
:100B60007461726174652028302D32293A2020206A
:100B700000352920486F70206368616E6E656C7364
:100B80003A2020202020003429204368616E6E65C1
:100B90006C2073706163696E673A202000332920EE
:100BA000524620706F7765722028302D37293A2001
:100BB0002020003229205246206D616769633A2067
:100BC0002020202020202020003129204261736530
:100BD000206672657175656E63793A202020000089
:100BE00000000700020100000304060000000000EE
:100BF00000000001020408102040800102040810D7
:100C00002001020408102004040404040404040263
:100C10000202020202030303030303000000002395
:100C2000002600290000000000250028002B0000FD
:100C3000000000240027002A0000622E11241FBE9D
:100C4000CFEFD8E0DEBFCDBF13E0A0E0B1E0E2ED32
:100C5000F2E602C005900D92A83CB107D9F716E064
:100C6000A8ECB3E001C01D92A239B107E1F71CE086
:100C7000CCE3DCE004C02297FE010E946B2FCA3354
:100C8000D107C9F70E949E2E0C9467310C94000086
:100C900080917705813019F482E080937705809107
:100CA0007705833019F484E0809377050895A8953B
:100CB0000895DC01ED91FC910190F081E02D099502
:100CC00008952091780530917905382748E0C901C9
:100CD000880F991F37FF06C09C0151E2252750E17C
:100CE000352701C09C01415091F73093790520933D
:100CF0007805089588E380937A0580E092ECA1E07E
:100D0000B0E080937B0590937C05A0937D05B09324
:100D10007E0587E08093870580E091EAACEBB3E342
:100D200080937F0590938005A0938105B093820501
:100D300085E0809388058DEE9EEFADEABEED809351
:100D4000830590938405A0938505B0938605E9E813
:100D5000F5E080E090E0863028F4DC01AE54BC4F32
:100D60002C9101C020E0219301968831910599F7DB
:100D700082E08093A1058AE08093A205089580E037
:100D80009EECADEEB4E38093BF059093C005A093B5
:100D9000C105B093C20580E090E0A0E0B0E580938B
:100DA000C3059093C405A093C505B093C605E7ECB1
:100DB000F5E080E081938F5F8031E1F70895A0E056
:100DC000B0E0E5EEF6E00C94342FD82F0E9499297C
:100DD0006115710581059105C9F30E94D72F109205
:100DE0008305109284051092850510928605C4E053
:100DF000812C912C54018A94C0908305D090840555
:100E0000E0908505F0908605FE2CED2CDC2CCC24A2
:100E10000E94D22FA50194010E94132F6C0D7D1DFD
:100E20008E1D9F1D609383057093840580938505B7
:100E300090938605C15001F7DD2309F450C009E8FD
:100E400015E0E801A12CB12C62E3C62ED12CE12CD7
:100E5000F12C8881882309F442C0B39419F40E94CC
:100E60007A063DC00E94D22FA70196010E94132F3F
:100E7000E1E0E60FA9E8B5E08A2F801B8A1520F48F
:100E80008D918E13F9CFE9CF2091880530E0A0E154
:100E9000B7E20E94AB2E9B01AC01AE2FB0E00E94E6
:100EA000BA2E40907F05509080056090810570902B
:100EB0008205640D751D861D971D4090BF055090DD
:100EC000C0056090C1057090C205461657066806B9
:100ED000790618F2E993A39488E1A812BACFCDB7A6
:100EE000DEB7E0E10C94502F8436910520F4BC016C
:100EF00080E090E017C09C018E3B910528F42A55B4
:100F00003109AAE0B0E00CC0823D910528F4245BD1
:100F10003109A4E6B0E004C02D5C3109A8E5B2E0D7
:100F20000E94AB2EA4E6B0E09B01AC010E94BA2E59
:100F3000089590E08C599F4F0E947407089561E0D6
:100F400086E00E94462A60E086E00E947F2A82E0D6
:100F50008093B00085E08093B10061E083E00E945F
:100F6000462A60E083E00E947F2A0895CF93DF93B2
:100F7000EC010097E9F061E086E00E947F2A9E0183
:100F800040E050E068E478EE81E090E00E94132FAA
:100F90002F3F31054105510529F020F02FEF30E0BA
:100FA00040E050E02093B3008091B000806107C022
:100FB00060E086E00E947F2A8091B0008F7E80935F
:100FC000B000DF91CF91089560E08EE00E94462A44
:100FD00061E08FE00E94462A61E080E10E94462A9B
:100FE00060E082E00E94462A61E084E00E94462A96
:100FF000089542E050E068E476E080E00E94C9286D
:101000000895E3E0F0E089E080935700E491E67012
:1010100081E0E63009F080E00895CF93DF93C82F98
:101020000E940108882381F0DFB781E08093760574
:10103000F8940E94570688E180936000C093600096
:10104000C1110E945706DFBFDF91CF9108958F92A3
:101050009F92AF92BF92CF92DF92EF92FF92CF9387
:10106000FC01C0A5EC2FE770F0E0E658FC4FA08132
:10107000B0E0C7FF03C024E130E002C02FE030E061
:10108000FC0197A183E1989FF0011124E25CFE4FDF
:1010900080809180A280B380A20FB31F20E43FE143
:1010A0004DE750E00E94C52EA50194010E94F12E4B
:1010B0008C2F887149F469017A01E0EDCE0EE7E0EA
:1010C000DE1EE11CF11C1BC0C7FF05C060E47AE80E
:1010D0008CE29EE004C060E07EEE8AEB9BE069015A
:1010E0007A01F8EBCF0EFBE0DF1EE11CF11CA5013D
:1010F00094010E94F12EC20ED31EE41EF51EC701FC
:10110000B60169517C4F8F4F9F4F28EE33E040E08E
:1011100050E00E94F12EA8EEB3E00E94BA2ECF91CB
:10112000FF90EF90DF90CF90BF90AF909F908F9007
:1011300008958F3F910551F048F0811522E0920704
:1011400038F08115934030F482E0089580E00895EE
:1011500081E0089583E00895A0E0B0E0E2EBF8E0DC
:101160000C943D2FEB018A01B82FB695A0E02881A1
:101170003981F80120832A813B8121832C813D81A3
:1011800022832E813F812383688179814A815B811B
:101190002C813D81EE81FF819F2F9295990F990FB0
:1011A000907C272F2370922B252F2370220F220F44
:1011B000922B232F23702295207F922BF80194836A
:1011C0000B5F1F4F2896AF5FBA1788F680FF24C0C9
:1011D000888199810E949908D82E8A819B810E94DA
:1011E0009908E82E8C819D810E949908F82E8E81A5
:1011F0009F810E949908F0E4DF9EA001112490E1F4
:10120000E99E90011124242B282BE4E0FE9EB001DE
:101210001124262BF8012083CDB7DEB7E7E00C942C
:10122000592F803223E0920708F1883E23E092078D
:1012300040F48F519340E4E096958795EA95E1F765
:101240000895803D27E0920718F48C5D934008953F
:10125000883928E0920768F4885C974074E0969596
:1012600087957A95E1F78D509C4F089580E090E046
:1012700008958FEF93E008958C30910540F4A4E039
:10128000880F991FAA95E1F7885D9C4F0895843FC8
:1012900023E0920718F484529C4F0895811524E0AE
:1012A000920740F48657934FF4E0880F991FFA9500
:1012B000E1F7089580E998E008959C013695279517
:1012C00025753575821B930B9C012373337396959B
:1012D00087959695879583739373820F931F9C01CF
:1012E00054E0369527955A95E1F7280F391F2F704E
:1012F0003F7041E051E0249FC001259F900D349F35
:10130000900D1124892F08954298882319F0000028
:10131000419A02C0000041980000429A00000895DE
:10132000429A000086B14298000081700895CF93E0
:10133000DF93D82F5C9A42985C98C8E08D2F807814
:101340000E948409DD0FC150C9F74298DF91CF9107
:1013500008958F770E9497090895CF93DF93D82F30
:10136000C8E08D2F80780E948409DD0FC150C9F735
:101370004298DF91CF910895CF93DF934298C8E0D0
:1013800080E0D82FDD0F0E9490098D0FC150C9F762
:10139000DF91CF9108950E94A9090E94BC095C9A2F
:1013A0000895A1E0B0E0E7EDF9E00C94422F8068E9
:1013B00069830E9497096981862F0E94AD095C9A12
:1013C0002196E2E00C945E2FCF93C0918305C8274D
:1013D000E82FF0E0E658FA4F678589E70E94D109C7
:1013E0006C2F8DE30E94D1096C2F82E40E94D109F9
:1013F000CF91089586E20E94CB090895CF93DF93A1
:10140000EC016C818CE10E94D1096D818DE10E941B
:10141000D1096E818EE10E94D1096F8180E20E9424
:10142000D109688581E20E94D109698582E20E9422
:10143000D1096A8583E20E94D1096B8584E20E940A
:10144000D1096C8585E20E94D1096D858AE20E94EE
:10145000D1096E858EE60E94D1096F858FE60E94C4
:10146000D109688980E70E94D109698981E70E94D2
:10147000D1096A8982E70E94D109DF91CF9108954D
:10148000CF92DF92EF92FF92CF93DF936B017C01BB
:10149000C11488E3D8068CE9E8068CE1F80628F543
:1014A000C701B60120E836E948E950E00E94F12E74
:1014B000E901689760E879E687E69FEF0E94CD2E04
:1014C0006C0D7D1D8E1D9F1DF2E0660F771F881F1E
:1014D000991FFA95D1F721E732E040E050E00E94F1
:1014E000F12EF22EE32E80E421C0C701B60120E0E8
:1014F0003DE241E351E00E94F12EE901689760E08E
:1015000073ED8EEC9EEF0E94CD2E6C0D7D1D8E1D19
:101510009F1D660F771F881F991F21E732E040E06B
:1015200050E00E94F12EF22EE32E80E66C2F6F71B8
:10153000680F85E70E94D1096E2D86E70E94D109C8
:101540006F2D87E70E94D109DF91CF91FF90EF9037
:10155000DF90CF900895682F8DE60E94D1090895FD
:101560008F929F92AF92BF92CF92DF92EF92FF92B3
:10157000CF93DF93D82F83E00E94CB09809375052A
:1015800084E00E94CB098093740560E086E00E94AD
:10159000D10961E087E00E94D1096FE789E00E94EC
:1015A000D10965E08AE00E94D10962E18BE00E94E6
:1015B000D10965E18CE00E94D1096DEF8DE00E94B8
:1015C000D10960E08EE00E94D109DD2319F08BE2A1
:1015D00091E008C02091A10533E1239FC0011124AF
:1015E000825C9E4F0E94FE096CE880E30E94D10954
:1015F0006FE082E30E94D10962E483E30E94D10993
:101600008091A20587FF02C064E101C06AE084E323
:101610000E94D1096AE285E30E94D1096DE286E366
:101620000E94D10964ED87E30E94D10960E088E35C
:101630000E94D10960E089E30E94D109D11109C05B
:10164000C0908305D0908405E0908505F0908605D4
:1016500007C0C5E9CC2EC1ECDC2EED2CCEEDFC2E66
:10166000CAE38F2C9924AA24BB24682D8C2F0E94B6
:10167000D109682D85E08C0F0E94D109FE2CED2C3C
:10168000DC2CCC24CF5FCE3361F76FEF83E40E9474
:10169000D1096FEF84E40E94D1096FEF85E40E94C5
:1016A000D1096FEF86E40E94D109DD2311F066E0D5
:1016B00002C0609187058DE60E94D10960E089E74C
:1016C0000E94D109609188058AE70E94D10960E0F3
:1016D00083E70E94D10960E084E70E94D109D1111B
:1016E00009C060917F05709180058091810590917E
:1016F000820504C060E071EA8CEB93E30E94400A2B
:10170000DF91CF91FF90EF90DF90CF90BF90AF909F
:101710009F908F90089561E087E00E94D10964E274
:101720008EE70E94D10963E088E00E94D10960E061
:1017300088E00E94D10965E087E00E94D10962E05B
:1017400085E00E94D10983E00E94CB098093750552
:1017500084E00E94CB0980937405089583E00E9481
:10176000CB098093750584E00E94CB0980937405B2
:1017700061E087E00E94D1096AE070E080E090E0DB
:101780000E94BC290E948B0B00000895CF92DF922B
:10179000FF920F931F93CF93DF931F92CDB7DEB7C6
:1017A000082F162F8EE399830E94D109F02EC02EA8
:1017B0009981D92E8C2D8F19811738F4F6016191FA
:1017C0006F018FE70E94D109F5CF64E085E00E94A8
:1017D000D10983E00E94CB098093750584E00E94C3
:1017E000CB09809374050E949929609370057093CA
:1017F0007105809372059093730569E087E00E94FC
:10180000D10981E0809377050F90DF91CF911F91EF
:101810000F91FF90DF90CF9008950F931F930E9438
:10182000C60B80917705813099F40E949929009127
:101830007005109171052091720530917305601B40
:10184000710B820B930B603A76488140910548F307
:1018500080917705813031F46EE971E086EE95E094
:101860000E94852B1F910F9108950F931F938091D4
:101870007705823021F41092770581E020C08091B5
:1018800077058130D9F40E94992900917005109153
:1018900071052091720530917305601B710B820BED
:1018A000930B613A76488140910540F061E087E012
:1018B0000E94D1091092770582E001C080E01F915B
:1018C0000F910895CF93DF93EC014AE050E06D2F24
:1018D00070E086EE95E00E94532C6EE286EE95E075
:1018E0000E94572BBE0184E0769567958A95E1F7B3
:1018F0006F7077274AE050E086EE95E00E94532C07
:101900006EE286EE95E00E94572BBE016F7077273E
:101910004AE050E086EE95E00E94532CDF91CF9193
:101920000895D82FC0E0CD1790F4439A299A64E621
:1019300070E080E090E00E94BC294398299864E61A
:1019400070E080E090E00E94BC29CF5FECCF6CE2B9
:1019500071E080E090E00E94BC29E4CF0F931F93D8
:10196000CF93DF93EC01062F15E0115051F0CE011B
:101970000E944E31081741F0602FCE010E9456316F
:10198000F4CF82E00E94910CDF91CF911F910F91D3
:101990000895A0E0B0E0EFECFCE00C94342F482E6A
:1019A000562EC0E0D0E0612C712CE12CF12C00E02F
:1019B00010E041100CC06090D80586E4689E3001AC
:1019C000112459E1E52EF12C0EEB15E01EC091E03B
:1019D00049120FC06090D805E6E46E9E30011124D4
:1019E000FBE16F0E711C49E2E42EF12C0AE715E0D1
:1019F0000CC082E0481209C028E1622E772473945B
:101A0000EE24E394F12C07ED15E043018C0E9D1EAE
:101A100010927905109278053401A62CA818B12CE3
:101A2000C30101966C01AE14BF04A8F4A00EB11E50
:101A3000511006C0C3010E944E31F501808305C0DC
:101A4000F5016081C3010E94AE0CF50180810E9406
:101A500061063601E2CFC301511018C0C3010E94D4
:101A60004E31B82EC6010E944E312B2D30E0322F60
:101A70002227282B8091780590917905821793076A
:101A800079F4C0E0D0E05524539493CF36016091AF
:101A900079050E94AE0C60917805C6010E94AE0CDB
:101AA000C05EDE4FC13E92E0D90708F482CF852D9B
:101AB000CDB7DEB7E0E10C94502F61E082E00E94E8
:101AC000C90C089560E082E00E94C90C8091D7059E
:101AD000853020F01092D7050E945D0D8091D705CA
:101AE0008093D805089561E080E00E94C90C61E010
:101AF00081E00E94C90C089560E080E00E94C90C5A
:101B0000882351F060E081E00E94C90C882321F015
:101B100080917A05883349F00E94BF060E947A06B8
:101B200081E00E94DF060E94730D0895882319F05A
:101B30006AEA71E002C06EEA71E086EE95E00E940A
:101B4000852B0895FF920F931F93CF93DF9369EC3A
:101B50007BE086EE95E00E94312B40917F0550910D
:101B6000800560918105709182052AE030E086EE63
:101B700095E00E945A2C63EB7BE086EE95E00E9494
:101B8000312B4091830550918405609185057091BA
:101B9000860520E130E086EE95E00E945A2C6DE942
:101BA0007BE086EE95E00E94312B4AE050E06091A8
:101BB000870586EE95E00E94822C67E87BE086EE42
:101BC00095E00E94312B4AE050E06091880586EE56
:101BD00095E00E94822C61E77BE086EE95E00E9412
:101BE000312BC9E8D5E0F12C8E0188818823A9F03A
:101BF000FF2031F061EB71E086EE95E00E94542BFE
:101C000021964AE050E0F801608186EE95E00E945E
:101C10004B2CF394F8E1FF12E7CF86EE95E00E949B
:101C20005F2B6BE57BE086EE95E00E94312B4AE06E
:101C300050E06091A10586EE95E00E94822C66E45A
:101C40007BE086EE95E00E94312BE091A205E770E3
:101C5000F0E0EE0FFF1FEE57FC4F6081718186EEC2
:101C600095E00E94852B61E37BE086EE95E00E9483
:101C7000312B8091A2058871883069F028F4811198
:101C800013C068E27BE00CC0803141F0883161F420
:101C90006CE07BE005C06CE17BE002C066E17BE0CC
:101CA00086EE95E00E94732B68EF7AE086EE95E071
:101CB0000E94312B40917B0550917C0560917D0500
:101CC00070917E052AE030E086EE95E00E945A2C65
:101CD0006FED7AE086EE95E00E94312B8091C3058E
:101CE00080710E94960D66EC7AE086EE95E00E9487
:101CF000312B8091C30580740E94960D6DEA7AE0C5
:101D000086EE95E00E94312B8091C30580720E947F
:101D1000960D60E97AE086EE95E00E94312B8AE725
:101D200095E00E942708AB01BC012AE030E086EE76
:101D300095E00E943C2C6BE87AE086EE95E00E94EC
:101D4000312B8AE795E00E9427089B01AC0160E4F3
:101D500072E48FE090E00E94F12EBA01A9012AE01E
:101D600030E086EE95E00E943C2C68E87AE086EE52
:101D700095E00E94732BCDB7DEB7E5E00C945B2FA6
:101D80008F929F92AF92BF92CF92DF92EF92FF928B
:101D9000811107C06FE77AE086EE95E00E94732B11
:101DA0002FC090E00E94740724E630E040E050E04D
:101DB0000E94F12ECA01B9012AE030E040E050E073
:101DC0000E94F12E49015A016B017C012AE030E0AA
:101DD000B501A40186EE95E00E943C2C6EE286EEF1
:101DE00095E00E94572B2AE030E0B701A60186EE6D
:101DF00095E00E943C2C63E786EE95E00E94972BCD
:101E0000FF90EF90DF90CF90BF90AF909F908F901A
:101E100008951F93CF93DF9365E77AE086EE95E010
:101E20000E94312B8091A305813041F46CE57AE06A
:101E300086EE95E00E94732B10E050C0823019F4BA
:101E400065E47AE0F5CF843019F461E37AE0F0CF0D
:101E5000853091F766E27AE0EBCFC12FD0E0C93050
:101E6000D1050CF441C068E3610F86EE95E00E9455
:101E7000572B6EE17AE086EE95E00E94312BBE0191
:101E80006F5F7F4F4AE050E086EE95E00E941B2C8A
:101E900063E17AE086EE95E00E94312BCD55DA4F72
:101EA000E981E03218F566E07AE086EE95E00E947E
:101EB000312B8981803130F06DE673E086EE95E05C
:101EC0000E94542B69816F7070E06F5F7F4F4AE012
:101ED00050E086EE95E00E94242C1F5F80914C0517
:101EE000181708F4BACF0FC061E3BECFEF70F0E06F
:101EF000EE0FFF1FEE56FC4F6081718186EE95E07C
:101F00000E94852BEACF6BEE79E086EE95E00E9489
:101F1000312B8091BB050E94C00E60ED79E086EE0A
:101F200095E00E94312B8091BC050E94C00E65EBAC
:101F300079E086EE95E00E94312B8091BD050E94EC
:101F4000C00E6AE979E086EE95E00E94312B40915F
:101F5000B3055091B4056091B5057091B605411572
:101F600051056105710539F12AE030E086EE95E012
:101F70000E945A2C67E679E086EE95E00E94312BAC
:101F80008091B7050E949907AB01BC012AE030E0BF
:101F900086EE95E00E945A2C63E479E086EE95E0A7
:101FA0000E94312B4AE050E06091B80586EE95E042
:101FB0000E94822C06C06AE379E086EE95E00E94DA
:101FC000732B6DE179E086EE95E00E94312B6091F4
:101FD000B9057091BA054AE050E086EE95E00E949E
:101FE0006C2C60E079E086EE95E00E94312B6091E8
:101FF000B205603450F470E06F5F7F4F4AE050E00C
:1020000086EE95E00E94242C06C067EF78E086EE0D
:1020100095E00E94732B6AED78E086EE95E00E94D1
:10202000312B8091B10580FF03C063EB71E002C0EA
:1020300067EB71E086EE95E00E94852B6DEB78E012
:1020400086EE95E00E94312B8091B10582700E944E
:10205000960D6EE978E086EE95E00E94312B809136
:10206000B10584700E94960D6FE778E086EE95E0EA
:102070000E94312B8091B10588700E94960DDF91EE
:10208000CF911F9108950F931F93CF93DF932091CA
:1020900049052F3FA9F56FEF75E086EE95E00E94A8
:1020A000312B86E893E00E94620C6EED75E086EEBF
:1020B00095E00E94312B80914A0590914B050E943A
:1020C000620C6BEA75E086EE95E00E94732B68E87F
:1020D00075E086EE95E00E94732B60E775E086EE72
:1020E00095E00E94732B6BE475E086EE95E00E940C
:1020F000732B86EE95E00E945F2B0E94090F68C04B
:1021000012160CF065C0332727FD309580914C05E1
:1021100090E0821793070CF45BC066E375E086EEEF
:1021200095E00E94312B60914905772767FD7095F6
:102130004AE050E086EE95E00E94242C6BE075E0CA
:1021400086EE95E00E94312B10E008E280914D056B
:102150001817D0F5C12FD0E0CC0FDD1FC25BDA4FCE
:10216000288130E080914905992787FD9095019756
:102170002817390739F56BEB71E086EE95E00E9480
:10218000542B4AE050E0602F86EE95E00E944B2CE5
:102190006FEB71E086EE95E00E94542BE981EF70C1
:1021A000F0E0EE0FFF1FEE56FC4F6081718186EE6E
:1021B00095E00E94542B63EC71E086EE95E00E945E
:1021C000542B0F5F1F5FC2CF86EE95E00E945F2BFE
:1021D000DF91CF911F910F910895FF920F931F935D
:1021E000CF93DF93C9E8D5E0F12C8E018881882355
:1021F000D1F165EC71E086EE95E00E94542B4AE047
:1022000050E06F2D86EE95E00E944B2C62ED71E060
:1022100086EE95E00E94542B2196F801208130E053
:10222000A0E1B7E20E94AB2E9B01AC01A091880512
:10223000B0E00E94BA2EAB01BC0180917F05909165
:102240008005A0918105B0918205480F591F6A1F32
:102250007B1F2AE030E086EE95E00E945A2CF39432
:10226000F8E1FF12C2CFCDB7DEB7E5E00C945B2FEB
:102270001092E30485E6E4EEF4E0DF011D928A9516
:10228000E9F70895CF93C82F8F3719F0883009F0F8
:1022900045C0E091E304EE23D9F1E150E093E3047B
:1022A000F0E0EC51FB4F10826DE070E086EE95E0BF
:1022B0000E945906C0E08091E304C81760F4EC2F37
:1022C000F0E0EC51FB4F608170E086EE95E00E94FB
:1022D0005906CF5FF0CF60E270E086EE95E00E9495
:1022E00059066DE070E086EE95E00E945906C0E068
:1022F0008091E304C81778F5EC2FF0E0EC51FB4F28
:10230000608170E086EE95E00E945906CF5FF0CFC5
:1023100067E086EE95E00E94572B1DC08B3119F4C3
:102320000E9438111AC08D30C1F08A30B1F080910E
:10233000E304843668F76C2F70E086EE95E00E9427
:102340005906E091E30481E08E0F8093E304F0E00E
:10235000EC51FB4FC08380E001C081E0CF91089534
:10236000CF93C82F0E9499296093CC047093CD0419
:102370008093CE049093CF04C093E104CC2329F042
:1023800040E051EE60E070E004C040E855E260E0FB
:1023900070E086EE95E00E94E12DCF910895909136
:1023A000D004492F4F7050E0BA016F5F7F4F292F43
:1023B00030E0E4E035952795EA95E1F76217730779
:1023C00059F0FA01EF52FB4F808381E0890F8F7043
:1023D000907F892B8093D00408956EE770E086EE9D
:1023E00095E00E9459060895A3E1B1E0EAEFF1E11A
:1023F0000C94352FE9E8F5E0712C8191882321F0C8
:10240000739428E17212F9CF66ED71E086EE95E0E3
:102410000E94852B4AE050E0672D86EE95E00E94F1
:10242000822C80E00E94B00A0E948B0B8E010E5F0E
:102430001F4FC12CD12C7601C39466246A945C2C66
:102440000E948D294B015C012091880530E0A0E1BC
:10245000B7E20E94AB2E9B01AC01C701B6010E94FE
:10246000CD2E20917F0530918005409181055091BE
:102470008205620F731F841F951F2091BF05309145
:10248000C0054091C1055091C2052617370748077E
:10249000590718F4F80160822AC08C2D0E94E409C3
:1024A00061E070E080E090E00E94BC29F8011082B9
:1024B0000E948D29681979098A099B09643F714036
:1024C0008105910540F40E94FA09F801908198175E
:1024D00078F78083EDCF85B150FE05C08B7D85B93F
:1024E000439A299A04C0846285B9439829982FEFAA
:1024F000C21AD20AE20AF20A0F5F1F4F8FEFC81604
:10250000D104E104F10409F09ACFCE019395FC01C6
:10251000D82E7FEF68EC2E2F281B271510F051E0E6
:1025200056C0DE01129651E02FEF41E03D91321787
:1025300010F0322F01C0452F5F5F5F3F11F0232F56
:10254000F5CF4193242F30E0A1E0B0E0AC0FBD1FE8
:10255000A20FB31F5C93413079F0DE01A20FB31FCD
:102560005C93423049F0AFEFBFEFAC0FBD1FA20F3D
:10257000B31F6C934E3F78F6A2E0B0E0AC0FBD1FE6
:10258000A20FB31F7C934D3F30F6A3E0B0E0AC0F39
:10259000BD1FA20FB31F6C93BECF452F242F30E079
:1025A000FC01E20FF31F6081AFEFB0E0AC0FBD1F85
:1025B000A20FB31F2C91621748F44150DC01A40F05
:1025C000B11D2C9120836C934111E8CF5F5F5715AB
:1025D00020F3372D369520E0231770F4DC01A20F8D
:1025E000B11D4C91522F530FFC01E50FF11D50818D
:1025F0005C9340832E5FF0CFF9E8EF2EF5E0FF2EDD
:102600008C01802F8D19871598F4F801C1908F01E6
:102610004AE050E06C2D86EE95E00E944B2C6CE277
:1026200086EE95E00E94572BF701C1927F01E9CF1A
:1026300086EE95E00E945F2B81E0CD5EDE4FEFE0FD
:102640000C94512F1F920F920FB60F9211241F93CB
:102650002F933F934F935F936F937F938F939F93AA
:10266000AF93BF93CF93DF93EF93FF93C091860017
:10267000D091870080918704909188042091A904CB
:10268000211155C09E01281B390B8091C3059091E3
:10269000C405A091C505B091C60585FD02C036955B
:1026A0002795253C49E03407B8F140910A0150E0F4
:1026B00060E070E02CE1B695A795979587952A95EF
:1026C000D1F70097A105B10521F481E090E0A0E0E9
:1026D000B0E084179507A607B707D8F480910A01E0
:1026E0008F3FB9F040E080910A01481780F4842FB1
:1026F00090E0880F991FFC01E757FB4F2081318143
:10270000FC01E55FFE4F318320834F5FECCF1092D9
:10271000AA0410920A010BC02D3B82E0380720F07A
:1027200080910A018031D8F08FEF80930A01D09315
:102730008804C0938704FF91EF91DF91CF91BF91FF
:10274000AF919F918F917F916F915F914F913F9149
:102750002F911F910F900FBE0F901F901895109101
:102760000A0181E0810F80930A01C9010E941109C9
:10277000E12FF0E0EE0FFF1FE757FB4F91838083BF
:10278000D6CF83E0809380008AE980938100809196
:10279000C30586FD05C0809181008064809381001F
:1027A0008FEF9FEF909389008093880080916F0056
:1027B000806280936F000895CF93DF930E94620D33
:1027C0008091D805843039F58BE00E94B22AC1E0AF
:1027D000D0E0892B11F4C0E0D0E08CE00E94B22A56
:1027E000892B19F082E090E002C080E090E08C2B11
:1027F0009D2B8230910539F08330910539F0019796
:1028000039F481E006C01092D80505C082E001C00D
:1028100083E08093D805DF91CF9108956F3018F051
:1028200086958058089589E0689F802D1124089529
:10283000A0E0B0E0EEE1F4E10C943C2FC82F0E9440
:102840009929009138041091390420913A0430916B
:102850003B046B017C01C01AD10AE20AF30A97011A
:10286000860149E8C41643E1D406E104F10410F0FE
:1028700010923C04609338047093390480933A04B6
:1028800090933B042091A9048FEF820F8230E8F5EA
:10289000E0913C04EE2309F46EC1E13011F482E0D2
:1028A000D8C1E03178F581E08E0F80933C04F0E0F0
:1028B000E757FB4FC083803109F0D4C1EBE8F4E067
:1028C000213029F4A181A695A695808108C0808138
:1028D0009181A92FA695A695A69596958795A03145
:1028E00048F4B0E090E0AA0FBB1FA55FBE4F119661
:1028F0009C938E931092AA04329684E0E939F807EB
:10290000F9F6B0C110923C04ADC1233009F023C1E7
:10291000E0913C04E11118C0CF3009F011C10E94D0
:102920008D290091B7041091B8042091B904309119
:10293000BA04601B710B820B930B62307105810529
:10294000910508F089C1FCC0E73148F481E08E0FA1
:1029500080933C04F0E0E857FB4FC083F1C0E731BF
:1029600009F0ECC0C111EAC040E050E0ABE0CA01A0
:10297000B3E0880F991FBA95E1F7A49F9001A59F36
:10298000300D1124F901E757FB4F6081E1817E2F63
:10299000777075956795FC01EE0FFF1FE55FFE4FA1
:1029A00071836083F901E657FB4FB081B695B69508
:1029B000B695E181FE2FF295FF0FF07E6F2F6B2B06
:1029C000E695E695E6957E2F777075956795FC01FF
:1029D000EE0FFF1FE35FFE4F71836083F901E55740
:1029E000FB4FB081B295B695B695B370C181DC2F1F
:1029F000DD0FDD0F6D2F6B2BC295C695C695C3708D
:102A0000E281E170EE0FEE0F7E2F7C2B75956795BE
:102A1000FC01EE0FFF1FE15FFE4F71836083F90140
:102A2000E357FB4FB081B695E181FE2FF795FF2765
:102A3000F7956F2F6B2BE6957E2F777075956795C1
:102A4000FC01EE0FFF1FEF5EFE4F71836083F90103
:102A5000E257FB4FB081B295BF70E181FE2FF29536
:102A6000F07F6F2F6B2BE295EF707E2F777075954F
:102A70006795FC01EE0FFF1FED5EFE4F71836083D3
:102A8000F901E157FB4FB081BB1FBB27BB1FC181C1
:102A9000DC2FDD0F6D2F6B2BCC1FCC27CC1FE281E1
:102AA000E370EE0F7E2F7C2B75956795FC01EE0F82
:102AB000FF1FEB5EFE4F71836083F901EF56FB4F02
:102AC000B081B695B695E181FE2FF295FF0FFF0F0D
:102AD000F07C6F2F6B2BE695E6957E2F77707595C2
:102AE0006795FC01EE0FFF1FE95EFE4F7183608367
:102AF000F901EE56FB4F20812295269527703181F2
:102B0000E32FEE0FEE0FEE0F6E2F622B732F7295E9
:102B10007695777075956795FC01EE0FFF1FE75E60
:102B2000FE4F718360834F5F5F4F4230510509F064
:102B30001ECF80919F0483FF1092AA0410923C0440
:102B40000E948D296093B7047093B8048093B904F0
:102B50009093BA0487C0243009F084C060913C048B
:102B600061110BC0C83AB1F4109279051092780542
:102B700088EA0E94610681E06CC0613019F4C0935C
:102B8000370404C0623031F4C09336048C2F0E94A5
:102B900061065AC0E09136042E2F30E0220F331F19
:102BA000462F50E0C9010296841795073CF0633226
:102BB00068F7FA01EA57FB4FC083E8CF2D5F3F4F1C
:102BC0008C2F90E06091780570917905421753073A
:102BD00049F4982F88278627972790937905809323
:102BE000780532C06817790769F58091370481301C
:102BF00049F5E13118F080E180933604F090360415
:102C0000CAE8D4E000E010E00F15D0F4FE013197DF
:102C1000808190E0982F88272881822B63E0969509
:102C200087956A95E1F70E941109F801EE0FFF1FE1
:102C3000E55FFE4F918380830F5F1F4F2296E4CFA5
:102C40001092AA0410923C0480913C04882351F015
:102C50008F5F80933C0406C080913C048F5F80931B
:102C60003C046ECFCDB7DEB7E8E00C94582FCF937D
:102C7000DF93E82FF0E0E254FA4FE185E03150F4C1
:102C8000F894F0E0EE0FFF1FE55FFE4F8081918129
:102C900078945DC08EE08E0F8B3058F4F0E0E25FE8
:102CA000F10924E62E9FC0012F9F900D11240C9650
:102CB0004EC0E03F09F446C038F4E13181F0E23122
:102CC00091F0E03139F409C0ED3FB1F1EE3FB9F1D7
:102CD000E13F79F180E092E03AC082E101C083E116
:102CE0000E94DB2A34C08BE00E94B22AC1E0D0E00F
:102CF000892B11F4C0E0D0E08CE00E94B22A892B2D
:102D000019F082E090E002C080E090E08C2B9D2BD7
:102D10008230910541F08330910541F00197A9F08F
:102D200086EA92E014C08CE090E011C089E591E061
:102D30000EC086E090E00BC08AEF93E008C08FEFF2
:102D400093E005C080E090E002C084EF93E0DF9163
:102D5000CF910895A2E2B0E0E0EBF6E10C94322FBF
:102D60009E012F5F3F4F80E1D9011D928A95E9F7BF
:102D700064E072E086EE95E029A33AA30E94852BD9
:102D80000E94AE0B1D8A1E8A1F8A188E312C212CA0
:102D900000E0812C912C5401412C74E7572E7BE8E4
:102DA000672E72E3772EE0E5CE2EE3ECDE2EE12CEB
:102DB000F12C84EF91E0A0E0B0E08D8F9E8FAF8F7B
:102DC000B8A380E09EECADEEB4E3898F9A8FAB8F11
:102DD000BC8F80E094E7ABE8B2E3898B9A8BAB8B36
:102DE000BC8B86EE95E00E94992C892B09F4E1C0FA
:102DF00086EE95E00E94C62C9C0133272C323105CB
:102E000009F442C0ACF42332310509F0ABC0198299
:102E10001A821B821C821D821E821F8218861986BE
:102E20001A861B861C861D861E861F86188A60C011
:102E30002434310529F02335310509F4B2C092C09C
:102E400064E486EE95E00E94572B2AE030E040E0F3
:102E500054E76BE872E386EE95E00E94E52B6CE2A6
:102E600086EE95E00E94572B2AE030E040E05EECD1
:102E70006DEE74E386EE95E00E94E52B6CE286EE43
:102E800095E00E94972BADCF0F5F043009F0A9CFDA
:102E900029813A814B815C81A8EEB3E00E94BA2E71
:102EA000698B7A8B8B8B9C8B2D813E814F815885D2
:102EB0000E94BA2E698F7A8F8B8F9C8F29853A85D5
:102EC0004B855C852D8F3E8F4F8F58A32D853E857A
:102ED0004F8558890E94BA2E6B017C0160323EE416
:102EE00073078105910530F462E38CE10E94D109FA
:102EF00000E077CF603345E774078105910510F452
:102F000062E2F3CF60345CE975078105910510F446
:102F100066E2EBCF80E5C81683ECD806E104F10445
:102F200010F462E1E2CF90E6C9169AEED906E10408
:102F3000F10410F465E1D9CFA0E7CA16A1E1DA06E1
:102F4000A1E0EA06F10410F461E0CFCFB0EACB16BD
:102F5000B6E8DB06B1E0EB06F10410F463E0C5CFA0
:102F600065E0C3CF10ED180F1A3008F03ACFE1E05A
:102F7000F0E0EC0FFD1F24E0029FE00DF11D112495
:102F80002081318142815381AAE0B0E00E94BA2EB3
:102F9000610F711D811D911D6083718382839383F5
:102FA00020CF49885A886B887C88812C912C5401C9
:102FB00018CF81149104A104B10489F4C301B201B2
:102FC0000E94400A61E070E080E090E00E94BC292D
:102FD0001D8A1E8A1F8A188E312C22242A948D8DD8
:102FE0009E8DAF8DB8A188169906AA06BB06D0F4AF
:102FF0000E94FA092D893E894F89588D280F311D6D
:10300000411D511D2D8B3E8B4F8B588F381608F468
:10301000382E821508F4282E3FEF831A930AA30A4C
:10302000B30A56C0C301B20128EE33E040E050E0DD
:103030000E94F12EBA01A9012AE030E086EE95E067
:103040000E943C2C6CE286EE95E00E94572B4AE0F1
:1030500050E0632D86EE95E00E944B2C6CE286EEEC
:1030600095E00E94572B6D897E898F89988DA501E7
:1030700094010E94F12EBA01A9012AE030E086EE07
:1030800095E00E943C2C6CE286EE95E00E94572B66
:103090004AE050E0622D86EE95E00E944B2C6CE2F7
:1030A00086EE95E00E94972B4C0C5D1C6E1C7F1CDD
:1030B000898D9A8DAB8DBC8D84159505A605B705B8
:1030C00020F449885A886B887C88812C912C540183
:1030D00029893A894B895C89283E3340410551054D
:1030E00009F07FCEA296E2E10C944E2FACE1B0E065
:1030F000ECE7F8E10C943C2F0E9499296B017C01CC
:1031000081E00E94B00A14E703E0198361E0CE0178
:1031100001960E940D0C009377050E948B0B6AEFBD
:1031200070E080E090E00E94BC29809177058330B8
:1031300089F486EE95E00E94992C892B59F40E941F
:1031400099296C197D098E099F096038734C894C47
:103150009140D8F280917705833009F44FC08FE712
:103160000E94A9090E94BC098983843511F083E07B
:103170005CC00E94BC0910924A0580934B050E94D6
:10318000BC0920914A0530914B05280F311D309321
:103190004B0520934A050E94BC0980934C050E9470
:1031A000BC0980934D05813110F7F12C0F2D10E0F3
:1031B00080914D0590E0880F991F0817190740F47A
:1031C0000E94BC09F801E25BFA4F8083F394EECFD2
:1031D00080E7898361E0CE0101960E940D0C83E0B7
:1031E000809377050E948B0B62E370E080E090E0B3
:1031F0000E94BC2980917705833011F482E015C0CC
:103200008FE70E94A9090E94BC098983803509F0D3
:10321000AECF03EA15E00E94BC09F80181938F014B
:10322000F5E00E3B1F07B9F781E06C96E8E00C94DF
:10323000582F80914905992787FD9095A92FB92F7F
:10324000FC013196EB30F10508F066C0EC5CFF4FF5
:103250000C94692F62E778E086EE95E00E94732B6C
:1032600086E893E00E94620C6AE578E086EE95E0DD
:103270000E94732B65E378E086EE95E00E94732B45
:103280006BE078E086EE95E00E94732B6AEE77E0C3
:1032900086EE95E00E94732B6DEB77E086EE95E06D
:1032A0000E94732B67E977E086EE95E00E94732B0E
:1032B00063E777E086EE95E00E94732B6CE477E09D
:1032C00086EE95E00E94732B86EE95E00E945F2BC0
:1032D0000E94A20D21C06FE277E01AC06AE077E099
:1032E00017C065EF76E014C066ED76E011C062E9C4
:1032F00076E00EC06DE776E00BC068E676E086EE1D
:1033000095E00E94732B62E276E002C06CE076E00A
:1033100086EE95E00E94732B6AE070E080E090E01A
:103320000E94BC2986EE95E00E94992C892B29F0F9
:1033300086EE95E00E94C62CF5CF0895ACE1B0E092
:10334000E4EAF9E10C943C2F909149059F3F09F084
:1033500023C1482F50E0FA013A97EF36F10508F003
:103360000FC1E15CFF4F0C94692F61E172E0A0C0D6
:103370006DE172E086EE95E00E94852B85E78983FA
:103380008BE1E3EAF5E0DE01129601900D928A9559
:10339000E1F76CE1CE0101960E940D0C0E948B0BAF
:1033A00083E08093770568EC70E080E090E00E9415
:1033B000BC2980917705843009F0E2C08FE70E9434
:1033C000A9090E94BC098983853509F0D9C06DEE31
:1033D00074E086EE95E00E94732B6FEC74E086EE4D
:1033E00095E00E94732B61EB74E096C065E372E098
:1033F00086EE95E00E94852B89E6898361E0CE0107
:1034000001960E940D0C0E948B0B83E08093770540
:1034100068EC70E080E090E00E94BC298091770524
:10342000843009F0ADC08FE70E94A9090E94BC0951
:1034300089838E010E5F1F4F7E014DE1E40EF11C6A
:103440000E94BC09F80181938F01EE15FF05C1F7B9
:103450008BE1FE013296A3EAB5E001900D928A95C8
:10346000E1F78981893409F08BC063E974E086EE65
:1034700095E00E94732B65E774E086EE95E00E946C
:10348000732B67E574E048C06FE472E086EE95E068
:103490000E94852B8EEF8093490572C08052875021
:1034A000805390914C05981708F066C06EE572E065
:1034B00086EE95E00E94852B63C084E180934905E8
:1034C00060E274E029C085E18093490569EE73E00C
:1034D00023C086E18093490562EB73E01DC087E15C
:1034E0008093490568E673E017C088E18093490539
:1034F00067E573E011C089E18093490563E473E0F7
:103500000BC08AE1809349056EE273E005C08BE150
:103510008093490566E073E086EE95E00E94732B88
:103520002FC06CEE72E086EE95E00E94732B8091C6
:10353000B10591E01DC066ED72E086EE95E00E9457
:10354000732B8091B10592E013C061EC72E086EEBE
:1035500095E00E94732B8091B10594E009C066EA62
:1035600072E086EE95E00E94732B8091B10598E0A1
:1035700089278093B1058FEF809349050E944310FE
:1035800086EE95E00E94992C892B09F45AC186EEAB
:1035900095E00E94C62CF4CF0E944211882309F4C2
:1035A00050C18091E304811104C08FEF80934905DD
:1035B00040C140E050E060E070E084EE94E00E94A2
:1035C000E02F40914905042F112707FD1095212F69
:1035D000312FF8013197EB31F10508F01AC1E255AE
:1035E000FF4F0C94692F552747FD509520914C05AE
:1035F00030E0241735070CF40CC18B019C010150FD
:10360000110921093109003211052105310558F050
:10361000C0904D05EFE4F5E0F12CD12CA8E2EA2EA4
:10362000415051090FC0FA01ED55FA4F61506083C6
:10363000D8C0DF0111972C9130E02417350729F00D
:10364000F3943296FC10F5CFCAC00E2D10E020E0A6
:1036500030E0061717072807390741F42081DA01FF
:10366000AD55BA4F11962C93DD24D394E394E8CF53
:103670006F3F71058105910511F008F0CAC0609394
:10368000BB05AFC06F3F71058105910511F008F0D2
:10369000C0C06093BC05A5C06F3F71058105910551
:1036A00011F008F0B6C06093BD059BC02091E40402
:1036B00020622037E9F440E050E060E070E085EE01
:1036C00094E00E94E02F9B01AC01DC01CB0101974B
:1036D000A109B1090897A105B10508F0ADC0A4ED95
:1036E000B0E30E94BA2E6A5E7C4A8A46954E24C098
:1036F0002636E9F440E050E060E070E085EE94E0CA
:103700000E94E02F9B01AC01DC01CB010197A109D4
:10371000B1090797A105B10508F08EC0A8EAB1E686
:103720000E94BA2E645E7C438E46944E05C061159D
:1037300071058105910571F08B019C0114572B488F
:1037400032430130FAE51F07F2E62F07F2E03F07A8
:1037500008F05FC06093B3057093B4058093B5051E
:103760009093B6053EC06F3F71058105910511F03C
:1037700008F04FC06093B70534C08B019C01015025
:103780001109210931090F3F11052105310508F003
:1037900040C06093B80525C08B019C01045C1940B2
:1037A000210931090D344DE114072105310528F4B3
:1037B0007093BA056093B90514C061157105810550
:1037C000910521F48FEF8093B2050BC06134710530
:1037D00081059105F0F461506093B20502C0DD20CF
:1037E000C1F08091E20481111AC08091830590910B
:1037F0008405A0918505B09186050196A11DB11D96
:103800008093830590938405A0938505B0938605E6
:1038100006C060E772E086EE95E00E94852B0E946C
:1038200038118FEF809349056AE086EE95E00E949B
:10383000972B0E94431005C061E070E080E090E0AB
:103840007BCF6C96E8E00C94582F6AE572E086EE28
:1038500095E00E94732B62E472E086EE95E00E9490
:10386000732B86EE95E00E94992C892B31F086EE21
:1038700095E00E94C62C0E949E190E947618823004
:1038800029F0833051F46DE072E002C064E272E02E
:1038900086EE95E00E94732B08958FEF8093490583
:1038A0001092E2040E944310809149058E3F69F016
:1038B00086EE95E00E94992C892BB1F386EE95E077
:1038C0000E94C62C0E949E19EFCF08950F931F935C
:1038D000109149051F3F09F0D2C0893409F457C03F
:1038E00000F5883309F469C058F4803309F477C0CF
:1038F00008F061C08B3109F440C08132B1F1B9C028
:10390000813409F487C030F4893309F466C0803407
:1039100061F1AFC0823409F48EC0863409F448C026
:10392000A8C0823609F487C078F4883531F128F4CC
:103930008235C1F18335E1F09CC08A3509F494C029
:10394000813609F467C095C0823761F128F4863664
:1039500079F18936E1F08DC0883779F08A3709F43A
:1039600083C0833709F085C003C061E172E015C0F0
:103970000E94730D6EE872E004C00E947C0D68EA3C
:1039800072E086EE95E00E94852B8EEF70C00E945B
:103990007A060E94BF0667EC72E086EE95E00E9410
:1039A000852B67C081E00E94DF0660EE72E0F5CFF4
:1039B0000E94ED105EC080535AC06AEF71E086EE3F
:1039C00095E00E94732B9091A20588E0890F887181
:1039D000977E892B8093A2051AC089E048C067EEC4
:1039E00071E086EE95E00E94732B8091C305909163
:1039F000C405A091C505B091C60520E1822780933A
:103A0000C3059093C405A093C505B093C605109354
:103A100049052FC061ED71E086EE95E00E94732BA1
:103A20008091C3059091C405A091C505B091C605CC
:103A300040E4842710C060EC71E086EE95E00E94BF
:103A4000732B8091C3059091C405A091C505B091D9
:103A5000C60520E282278093C3059093C405A093F6
:103A6000C505B093C60502C00E94251C8FEF809348
:103A70004905809149058E3F09F0D4C0DDC00E9400
:103A80004211882309F4D8C08091E304811104C055
:103A90008FEF80934905C6C040E050E060E070E0E1
:103AA00084EE94E00E94E02F00914905112707FD64
:103AB0001095212F312FF8013197E930F10508F0E9
:103AC000B4C0E753FF4F0C94692F8B019C01015048
:103AD00014472B4832430F3F19452246324008F025
:103AE000A4C060937F0570938005809381059093B7
:103AF000820577C060938305709384058093850564
:103B00009093860581E08093E2046BC06830710574
:103B10008105910508F089C06093870562C08B011B
:103B20009C0101501109210931090A3011052105B3
:103B3000310508F07AC06093880553C061EB71E0ED
:103B400084EE94E00E941A3110E0009799F00E94F0
:103B5000F430009779F0183130F4E12FF0E0E658B6
:103B6000FA4F87871F5F61EB71E080E090E00E9471
:103B70001A31EBCF1831A8F5E12FF0E0E658FA4FF3
:103B800017861F5FF7CF653071058105910508F035
:103B90004CC06093A10525C08B019C010150110907
:103BA000210931090630110521053105F0F5209173
:103BB000A205287F262B2093A20513C08B019C0110
:103BC00001501109210931090115124C214031051B
:103BD00060F560937B0570937C0580937D059093E1
:103BE0007E058091E204811113C08091830590913C
:103BF0008405A0918505B09186050196A11DB11D92
:103C00008093830590938405A0938505B0938605E2
:103C10000E9438118FEF809349056AE086EE95E0A7
:103C20000E94972B0E94191907C060E772E086EE88
:103C300095E00E94852BECCF1F910F9108958FEF97
:103C4000809349051092E2040E9419198091490558
:103C50008E3F69F086EE95E00E94992C892BB1F396
:103C600086EE95E00E94C62C0E94661CEFCF6AE0AB
:103C700070E080E090E00E94BC2986EE95E00E9412
:103C8000992C892B29F086EE95E00E94C62CF5CF61
:103C90000895CF93C82F682F86EE95E00E94F32CED
:103CA00090916E059C2790936E05CF910895A1E0A9
:103CB000B0E0EDE5FEE10C94422F99830E94491E8D
:103CC0009981892F0E94491E2196E2E00C945E2F73
:103CD0001F93CF93DF93182FEB0110926E0565EBC6
:103CE00070E086EE95E00E94590662E670E086EE8E
:103CF00095E00E945906812F0E94491ECE010E9424
:103D0000571EDF91CF911F91089560916E0586EE49
:103D100095E00E94F32C0895A1E2B0E0E2E9FEE113
:103D20000C943E2F7B018A018C3009F453C108F0BA
:103D300040C0863009F4BCC018F5833009F491C046
:103D400070F4813009F472C0823009F04AC26BE12C
:103D500070E082E00E94681E03EA15E078C08430BB
:103D600009F487C0853009F03CC260914D0570E0D0
:103D7000660F771F85E00E94681E0EE415E086C07E
:103D8000893009F4A7C070F4873009F49BC08830EB
:103D900009F027C261E070E088E00E94681E80910F
:103DA000D80525C28A3009F4CAC08B3009F4F2C0A4
:103DB00018C28A3609F475C1D8F4873609F43AC1B5
:103DC00038F4853609F40EC1863609F41FC109C2DC
:103DD000883609F437C1893609F003C261E070E022
:103DE00089E60E94681E0E947A060E94BF06F7C1FB
:103DF0008D3609F4D4C138F48B3609F491C18C3670
:103E000009F49AC1EEC18E3609F4DEC1873C09F08F
:103E1000E8C161E070E087EC0E94681E81E00E94CA
:103E2000491E0E94851E10926F05E5C169E270E08F
:103E300081E00E94681E0AE715E0F80181918F0178
:103E40000E94491EF5E0033A1F07B9F7D2C1F801F5
:103E500081918F010E94491EF5E00E3B1F07B9F7C3
:103E6000C8C161E070E083E00E94681E0E9476187D
:103E7000BEC161E070E084E00E94681E81E00E94A3
:103E8000491E0E94851E0E94AA16B5C180914D054B
:103E900090E0880F991F98012E5435402817390754
:103EA00008F0A7C1F80181918F010E94491EEECF51
:103EB00062E070E086E00E94681E86E893E00E945F
:103EC000571E97C161E070E087E00E94681E8091F4
:103ED0004C058DC186E6898361E0CE0101960E9482
:103EE0000D0C0E948B0B83E08093770568EC70E0EB
:103EF00080E090E00E94BC29809177058430D9F45D
:103F00008FE70E94A9090E94BC098983863469F45D
:103F100060E270E089E00E94681E10E20E94BC0925
:103F20000E94491E1150D1F764C161E070E089E040
:103F30000E94681E54C161E070E089E055C169E1EA
:103F400070E08AE00E94681E81E08093BE052091A7
:103F500076058091C3059091C405A091C505B091E7
:103F6000C605222311F0806801C08F778093C305B6
:103F70009093C405A093C505B093C6050EEB15E05C
:103F8000F80181918F010E94491EF5E0073D1F074E
:103F9000B9F72FC161E270E08BE00E94681E80914A
:103FA000AA048F3F39F08091AA0491E0980F909372
:103FB000AA0402C08091AA040E94491E10E0812F29
:103FC0000E9437160E943C090E94571E1F5F103145
:103FD000B1F70FC161E070E08CE00E94681E809133
:103FE000D70505C161E070E085E60E94681E89E2A0
:103FF000E816F10409F0FAC0D801EAE7F5E08D917E
:10400000819385E0E33AF807D1F7E9C061E070E019
:1040100086E60E94681EEBE1EE16F10409F0E6C0A8
:10402000D801E3EAF5E08D91819385E0EE3BF80756
:10403000D1F7D5C061E070E087E60E94681E0E945B
:10404000730DCDC061E070E088E60E94681E85E7D0
:1040500089838BE1E3EAF5E0DE01129601900D928F
:104060008A95E1F76CE1CE0101960E940D0C0E9449
:104070008B0B83E08093770560E273E080E090E053
:104080000E94BC2980917705843009F0AFC08FE78A
:104090000E94A9090E94BC098983853509F0A6C040
:1040A0009EC061E070E08AE60E94681E89E689830E
:1040B00061E0CE0101960E940D0C0E948B0B83E003
:1040C0008093770560E273E080E090E00E94BC2975
:1040D00080917705843009F089C08FE70E94A90993
:1040E0000E94BC0989838E010E5F1F4F7E01EDE1A6
:1040F000EE0EF11C0E94BC09F80181938F01EE15B0
:10410000FF05C1F78BE1FE013296A3EAB5E001900D
:104110000D928A95E1F78981893409F067C05FC003
:1041200061E070E08BE60E94681EF8018081809358
:10413000D8050E947C0D53C061E070E08CE60E94BF
:10414000681EF0E2EF16F10461F487E6898380E2ED
:10415000F801DE01129601900D928A95E1F761E275
:1041600003C087E4898361E0CE0101960E940D0CB3
:104170000E948B0B83E0809377056CE474E080E011
:1041800090E00E94BC2980917705843079F58FE713
:104190000E94A9090E94BC09873441F520C061E052
:1041A00070E08DE60E94681E89E1E816F104F1F4E2
:1041B000D801EEEBF5E08D91819385E0E73DF807BE
:1041C000D1F70E94C1130BC061E070E08EE60E943F
:1041D000681EF80180818093D7050E945D0D81E003
:1041E00006C061E070E08AEC0E94681E80E00E94D8
:1041F000491E0E94851EA196E6E00C945A2FA0E06D
:10420000B0E0E5E0F1E20C943C2FCAECD3E014E618
:1042100006E035E0F32E44E0E42E53E0D52E62E0D4
:10422000C62E86EE95E00E94992C892B09F49BC03E
:1042300086EE95E00E94C62C282F8093350440918D
:10424000340450E04730510560F7FA01EE52FF4F59
:104250000C94692F853B29F781E080933404E1CFEA
:10426000823609F07DC0C0923404DBCF80933304E2
:1042700080933204D0923404D4CF9C0133273093FE
:1042800031042093300490913204982790933204A3
:10429000E0923404C6CF382F222740913004509149
:1042A0003104242B352B309331042093300490912A
:1042B0003204982790933204F09234042536310565
:1042C00008F4AFCF61E070E08CEC0E94681E81E0E2
:1042D0000E94491E0E94851E43C020912E043091E9
:1042E0002F04F901E653FC4F808390913204982704
:1042F00090933204C901019690932F0480932E0469
:1043000020913004309131048217930708F489CF4B
:104310000093340486CF8091320482130BC06091E5
:104320002E0470912F044AEC53E0809133040E94D4
:104330008C1E0DC062E070E08BEC0E94681E8091C4
:1043400033040E94491E80916E050E94491EFE01A1
:10435000812F11928A95E9F710922F0410922E0462
:10436000109234045ECFCDB7DEB7E8E00C94582F3E
:1043700081E080936F0580916F05882349F086EE78
:1043800095E00E94992C892BB1F30E94FF20F3CF76
:104390000895AAE2B0E0EFECF1E20C943A2F0E940B
:1043A0008D296B017C0181E00E94B00A86EE95E0C8
:1043B0000E94992C892B29F086EE95E00E94C62C4C
:1043C000F5CF4398299811E072E6B72EE9E2AE2EB8
:1043D00003E00E948D296C197D098E099F09693CB3
:1043E000710581059105F0F11123E1F10E948D29FC
:1043F0006B017C0185B1846285B980ED97E00E94F4
:10440000B607B982EAE7F5E0DE0112968A2D01903F
:104410000D928A95E1F76AE2CE0101960E940D0C99
:1044200085B18B7D85B980E090E00E94B60700934E
:1044300077050E948B0B62E370E080E090E00E94C1
:10444000BC2980917705843061F4009377058FE76C
:104450000E94A9090E94BC0911E0823419F410E0FD
:1044600001C011E087E00E94B22A892BB1F411E06B
:1044700014C0439A299A85B1846285B986EE95E085
:104480000E94C62C8D309105C1F074F40A97A9F0F2
:104490004398299885B18B7D85B986EE95E00E9479
:1044A000992C892B31F795CF8332910579F082349D
:1044B000910571F70E94B821EBCF62EB71E086EEB7
:1044C00095E00E94732B0E941F1EE2CF0E94AA1645
:1044D000DFCF8F929F92AF92BF92CF92DF92EF92F7
:1044E000FF921F93CF93DF9387E00E94B22A892B1C
:1044F00009F089C068EC70E080E090E00E94BC297F
:1045000080E090E00E94B6070E948D294B015C017B
:104510006B017C0180ECC80E82E1D81EE11CF11C0D
:104520000E948D296C157D058E059F0530F487E06E
:104530000E94B22A892BA1F364C087E00E94B22AAC
:10454000892B09F05EC080ED97E00E94B6070E94BB
:104550008D296B017C01D0E0C1E088E4880E86E201
:10456000981EA11CB11C11E087E00E94B22A892B81
:1045700021F58C149D04AE04BF0430F480ED97E067
:104580000E94B607D1E0F0CF0E948D296C197D09F9
:104590008E099F09693C71058105910528F30E94E8
:1045A0008D296B017C01C12719F080ED97E002C0D5
:1045B00080E090E00E94B607D7CF80E090E00E94B4
:1045C000B607DD23B9F08091D70590E0019665E04C
:1045D00070E00E94DD2E8093D7050E945D0D0E9441
:1045E000DC130E947C0D64EF71E080E090E00E949B
:1045F000BC2909C080E00E94DF060E94F4110E94DD
:10460000730D0E94C921DF91CF911F91FF90EF9010
:10461000DF90CF90BF90AF909F908F900895CF92F2
:10462000DF92EF92FF9280E00E940D080E94E40763
:1046300061E081E10E94462A61E08DE00E94462A05
:1046400061E089E00E94462A61E08AE00E94462AF1
:1046500060E087E00E94462A60E08BE00E94462AE4
:1046600061E08BE00E947F2A60E08CE00E94462A95
:1046700061E08CE00E947F2A60E088E00E94462A88
:1046800061E088E00E947F2A0E949F0740E052EC90
:1046900061E070E086EE95E00E94E12D0E94DC135F
:1046A0000E947C0D0E94C1138FEF8093AA040E9488
:1046B000F90778940E948D296B017C018091AA04EE
:1046C0008F3F59F40E948D296C197D098E099F092D
:1046D000603D77408105910588F380ED97E00E9469
:1046E000B60761E087E00E947F2A439A299A86EE06
:1046F00095E00E94992C892B29F086EE95E00E9486
:10470000C62CF5CF6DEF72E086EE95E00E94542B3B
:1047100086E893E00E94620C64E173E086EE95E027
:104720000E94542B4AE050E063E070E086EE95E092
:104730000E94242C62E370E080E090E00E94BC299B
:1047400086EE95E00E94992C04970CF186EE95E098
:104750000E94C62C82349105D1F486EE95E00E9429
:10476000C62C8E34910599F486EE95E00E94C62CF5
:104770008434910561F486EE95E00E94C62C819701
:1047800031F480E090E00E94B6070E94C921409178
:104790007B0550917C0560917D0570917E05DB0164
:1047A000CA010197A109B1090497A105B10568F4EF
:1047B0004093A904433029F440EA56E861E070E0F0
:1047C00004C040E052EC61E070E086EE95E00E94AB
:1047D000E12D0E9469224398299880E090E00E9490
:1047E000B6070E94C1131092C9048091C30583FFCC
:1047F00011C080918F05882351F080919605882300
:1048000031F080919D05882311F087E001C085E09B
:104810008093C90480E00E94B00A8091CA040E947B
:10482000E4090E948B0B10923F0410923E041092F8
:104830003D04F12C8091D8058F15B0F062E370E053
:1048400080E090E00E94BC2980ED97E00E94B607CE
:1048500062E370E080E090E00E94BC2980E090E09C
:104860000E94B607F394E6CF8091A20584FF08C0AA
:10487000982F987181E0983109F080E00E94B01182
:104880008FE00E940D08FF90EF90DF90CF90089589
:10489000EF92FF920F931F93CF93DF938C016EE7FC
:1048A00070E086EE95E00E945906E801F12CF0E2F6
:1048B000EF2E8E0188818D57823048F46DE770E0CD
:1048C00086EE95E00E94590688818E258883219680
:1048D000F801608186EE95E00E94F32CF394F9E0F4
:1048E000FF12E7CF6EE770E086EE95E00E94590672
:1048F000CDB7DEB7E6E00C945A2FA9E0B0E0E3E8CC
:10490000F4E20C94422F9091CB0491110EC09EEFD3
:1049100099838A836B8350E0559547954C832D830B
:10492000198618861F821E822EC04091D004842FC3
:1049300090E0B4E095958795BA95E1F7242F2F7014
:1049400030E08217930719F18DEF89831B82FE01F6
:10495000349650E0842F90E0A4E095958795AA9531
:10496000E1F7242F2F7030E08217930749F0DC0124
:10497000AF52BB4F8C918193405F5F5F563051F7D0
:104980004093D0045A83CE0101960E94482480911E
:10499000CB0490E0019666E070E00E94DD2E8093EB
:1049A000CB042996E2E00C945E2FA0E0B0E0EBEDA2
:1049B000F4E20C943B2F6C016EE770E086EE95E01C
:1049C0000E9459068601E12CF12CC0E0D0E030E2D3
:1049D000B32EF801608183E8860F823078F46DE7AA
:1049E00070E086EE95E00E945906F80160816B2523
:1049F00070E086EE95E00E94590604C086EE95E0D0
:104A00000E94F32CE114F10459F0F80180819E0119
:104A1000280F311DC901C92FDD27C80FD91FDD2778
:104A20003FEFE31AF30A89E0E816F10459F028E0B1
:104A3000E216F10421F48C2F8095F60180870F5F38
:104A40001F4FC7CFCDB7DEB7E9E00C94572FA9E0D1
:104A5000B0E0EDE2F5E20C94422FE82F362F809182
:104A6000CB0490E0019664E270E00E94DD2E80931A
:104A7000CB0458E9598350E15A83813089F048F0DA
:104A80008230B9F08330D9F48B8381EF8C833D83FE
:104A900019C085E08B8381EF8C832F5F2D8312C03B
:104AA0008B8381EF8C8384E6489FA00111245D8372
:104AB00009C084E08B8381EF8C83ED8303C00E9467
:104AC000ED1104C0CE0101960E94D5242996E2E0A2
:104AD0000C945E2FA2E0B0E0E0E7F5E20C94372FF3
:104AE000182F762E2A8349830E9499296B017C0115
:104AF0008091E1048090CC049090CD04A090CE04ED
:104B0000B090CF042A8149818823C1F0D701C60122
:104B100088199909AA09BB094C015D0191EE891612
:104B20009EE29906A104B10420F1241708F4422F53
:104B3000202F672D812F0E94272513C0D701C60182
:104B400088199909AA09BB094C015D0191E38916ED
:104B500095E79906A104B10460F0672D812F0E94AA
:104B60007D24C092CC04D092CD04E092CE04F09289
:104B7000CF042296EDE00C94532FA2E2B0E0E3ECD8
:104B8000F5E20C94382F8CE00E94CB0981110FC004
:104B90006CE173E086EE95E00E94852B439A299A9A
:104BA00080E00E94B00A0E948B0B4398299886EE01
:104BB00095E00E94992C892B01F186EE95E00E94E8
:104BC000C62C9091A904992319F00E941814EFCFD4
:104BD00040913E0450E09A012F5F3F4F2F713327E1
:104BE00060913F0470E02617370709F3FA01E75B8D
:104BF000FB4F808320933E04DACF80917705843089
:104C000009F086C00E9499296115710581059105F9
:104C100049F06093BB047093BC048093BD049093EF
:104C2000BE040CC081E090E0A0E0B0E08093BB0443
:104C30009093BC04A093BD04B093BE048091AD04D6
:104C40009091AE0481609093AE048093AD0483E0B4
:104C5000809377058FE70E94A90909E614E00E9476
:104C6000BC09F80181938F01F4E002371F07B9F7FF
:104C70002091720480916904982F922796FF3BC07F
:104C800090E4922790937204982F98739833F1F4DC
:104C900010E0212F30E080916904877090E0821746
:104CA00093074CF11F5F2091A205812F90E0FC013A
:104CB000E759FB4F24FF04C080810E94CF11E9CF48
:104CC000608186EE95E00E94F32CE3CF8F7399F418
:104CD00080916A048093B60480916B048093B4043D
:104CE00080916C048093B30480916F0490E0909362
:104CF000AC048093AB0480913D04813019F482E0D0
:104D000080933D0480913D04833011F410923D0462
:104D10000E9499296B017C018091AF049091B004AD
:104D2000A091B104B091B2040097A105B105C9F0FA
:104D3000A7019601281B390B4A0B5B0BDA01C9014D
:104D4000883B9B40A105B10560F00E94FA09809361
:104D5000B5041092AF041092B0041092B1041092F6
:104D6000B2048091BF049091C004A091C104B0919D
:104D7000C20446015701881A990AAA0ABB0A8AE79F
:104D800095E00E94270886169706A806B90608F43B
:104D9000B3C0C092BF04D092C004E092C104F092AC
:104DA000C2040E9457068091AA048830A0F0809126
:104DB000C3059091C405A091C505B091C6055CE1FD
:104DC000B695A795979587955A95D1F7892B8A2BF4
:104DD0008B2B09F0CCC18091AA048F5F8093AA0429
:104DE0008091BB049091BC04A091BD04B091BE041D
:104DF0000097A105B105F1F0C81AD90AEA0AFB0A21
:104E00008AE795E00E9427086C157D058E059F05B1
:104E100008F01FC18091C30584FD04C080ED97E0B8
:104E20000E94B6071092BB041092BC041092BD04FD
:104E30001092BE0490917204907C909372045091F1
:104E40003E0480913F0420913D04581709F41EC18F
:104E5000223009F01BC1905890937204E091A20592
:104E6000E770F0E0E658FC4F6081693008F0F6C06A
:104E7000615040E04613F4C080933F0487E3840F01
:104E800090917204892B809372044093400483E0D4
:104E900080933D0485B1846285B910918705809126
:104EA000C904811142C18091C30582FD4AC1812F8D
:104EB0000E94AB0A8091CA040E94E409E091A20515
:104EC000E770F0E0E658FC4F608182E794E00E94D2
:104ED000C60B8091C30582FD3EC1E091CA04EF5F1D
:104EE000E093CA04E83109F43FC1F0E0E658FA4F14
:104EF0008785882309F438C10E94350C813069F513
:104F00008091A205887149F18091AD049091AE0421
:104F1000880F991F9093AE048093AD0483E0809333
:104F200077050E948B0B0E9499296093AF047093C0
:104F3000B0048093B1049093B204672B682B692B63
:104F400061F481E090E0A0E0B0E08093AF04909342
:104F5000B004A093B104B093B2048091A20584FF81
:104F60002BC08091BB049091BC04A091BD04B09172
:104F7000BE04892B8A2B8B2BF9F08091AD04909184
:104F8000AE048E7F0E945D09182F6091AB04809162
:104F9000B6040E940E14482F612F8091B50449A3D6
:104FA0000E940E140091D805282F49A16091B304E6
:104FB0008091B4040E946A2585B18B7D85B980916A
:104FC000C7048130C1F018F08230B1F1DEC087E053
:104FD0000E94B22A892B09F0D8C081E08093C704CF
:104FE0000E948D296093C3047093C4048093C50408
:104FF0009093C604CAC087E00E94B22A892B31F57B
:105000000E948D29C090C304D090C404E090C504D0
:10501000F090C6046C197D098E099F09693E7340A2
:105020008105910508F4B1C082E08093C70480ED4A
:1050300097E00E94B607A9C087E00E94B22A892B98
:1050400009F4A3C080E090E00E94B6071092C70464
:105050009CC080E090E00E94B607ECCE68E009CFEB
:10506000851709F409CF4F5F242F30E090E0F90154
:10507000EE58FB4FDC01A75BBB4F7C917083F901BD
:10508000E05CFB4F708301968F71F4CE2430B1F455
:105090002091400481E494E0A3E7B4E0FC013E2FBA
:1050A000381B321718F431913D93F9CF87E3820F03
:1050B00090917204892B80937204E9CE8091C70489
:1050C000823059F4916090937204439A299A8E0128
:1050D0000F5F1F4FF12CB80111C0439829988091A0
:1050E0003D04811103C081E080933D0480913D0423
:1050F000833069F784E080933D04E9CF8F2D69A365
:105100007AA30E943716F801819391938F01F3944B
:1051100069A17AA1F0E1FF12F1CF8091A20543E7E6
:1051200054E087700E94AC08B5CE112309F4BBCEC1
:105130009091C80421E0290F2093C8049813B3CE9E
:1051400020C08BE00E94B22A892B09F0B0CE439A8E
:10515000299A17E0ACCE8BE00E94B22A892B09F085
:10516000BCCE43982998B9CE1092CA04C5CE80917E
:10517000AA04883011F4439A299A89E08093AA04FA
:10518000BBCE1092C80411508ECEA296ECE00C94C7
:10519000542F8230E8F4E82FF0E0EE0FFF1FE752C3
:1051A000FA4F71836083813041F0809169008C7F78
:1051B000842B80936900E89A089580916900440FD8
:1051C000551F440F551F837F842B80936900E99AF4
:1051D00008951F920F920FB60F9211242F933F93B1
:1051E0004F935F936F937F938F939F93AF93BF93EF
:1051F000EF93FF938091D9059091DA05892B29F0DF
:10520000E091D905F091DA050995FF91EF91BF91F1
:10521000AF919F918F917F916F915F914F913F914E
:105220002F910F900FBE0F901F9018951F920F9205
:105230000FB60F9211242F933F934F935F936F9369
:105240007F938F939F93AF93BF93EF93FF9380913F
:10525000DB059091DC05892B29F0E091DB05F091CD
:10526000DC050995FF91EF91BF91AF919F918F91CF
:105270007F916F915F914F913F912F910F900FBE52
:105280000F901F9018951F920F920FB60F92112436
:105290002F933F938F939F93AF93BF938091DE059E
:1052A0009091DF05A091E005B091E1053091DD0519
:1052B00023E0230F2D3720F40196A11DB11D05C059
:1052C00026E8230F0296A11DB11D2093DD058093D2
:1052D000DE059093DF05A093E005B093E105809192
:1052E000E2059091E305A091E405B091E5050196F2
:1052F000A11DB11D8093E2059093E305A093E40501
:10530000B093E505BF91AF919F918F913F912F9100
:105310000F900FBE0F901F9018952FB7F8946091C3
:10532000DE057091DF058091E0059091E1052FBFCA
:1053300008953FB7F8948091E2059091E305A0911C
:10534000E405B091E50526B5A89B05C02F3F19F0EF
:105350000196A11DB11D3FBF6627782F892F9A2F77
:10536000620F711D811D911D42E0660F771F881F1E
:10537000991F4A95D1F70895CF92DF92EF92FF924D
:10538000CF93DF936B017C010E949929EB01C1143B
:10539000D104E104F10479F00E9499296C1B7D0B82
:1053A000683E7340A0F381E0C81AD108E108F10813
:1053B000C851DC4FECCFDF91CF91FF90EF90DF90A1
:1053C000CF900895789484B5826084BD84B581605F
:1053D00084BD85B5826085BD85B5816085BDEEE6FD
:1053E000F0E0808181608083E1E8F0E010828081DC
:1053F00082608083808181608083E0E8F0E080814A
:1054000081608083E1EBF0E0808184608083E0EB69
:10541000F0E0808181608083EAE7F0E08081846051
:1054200080838081826080838081816080838081AD
:10543000806880831092C1000895833081F028F441
:10544000813099F08230A1F008958630A9F087303C
:10545000B9F08430D1F4809180008F7D03C08091B9
:1054600080008F7780938000089584B58F7702C085
:1054700084B58F7D84BD08958091B0008F7703C07F
:105480008091B0008F7D8093B0000895CF93DF931B
:1054900090E0FC01ED50F44F2491FC01E95FF34FE3
:1054A0008491882349F190E0880F991FFC01E15D08
:1054B000F34FA591B4918B5D934FFC01C591D491AD
:1054C0009FB7611108C0F8948C91209582238C932A
:1054D000888182230AC0623051F4F8948C91322F73
:1054E000309583238C938881822B888304C0F89421
:1054F0008C91822B8C939FBFDF91CF910895A1E077
:10550000B0E0E5E8FAE20C94402F282F30E0F901F2
:10551000E152F44F8491F901ED50F44F1491F901E7
:10552000E95FF34F04910023C9F0882321F06983D8
:105530000E941D2A6981E02FF0E0EE0FFF1FEB5D56
:10554000F34FA591B4919FB7F8948C91611103C06A
:105550001095812301C0812B8C939FBF2196E4E09D
:105560000C945C2FCF93DF93282F30E0F901E152A8
:10557000F44F8491F901ED50F44FD491F901E95FB2
:10558000F34FC491CC2391F081110E941D2AEC2F7E
:10559000F0E0EE0FFF1FE55EF34FA591B4912C9163
:1055A0002D2381E090E021F480E002C080E090E0D3
:1055B000DF91CF9108958E3008F08E508770209142
:1055C0009D0190E4299F90011124822B80937C00FF
:1055D00080917A00806480937A0080917A0086FDC1
:1055E000FCCF809178002091790090E0922B089573
:1055F000A0E0B0E0EEEFFAE20C943C2F6C017A01EF
:10560000EB01E60EF71E00E010E0CE15DF0561F0BD
:105610006991D601ED91FC910190F081E02DC601D8
:105620000995080F191FF1CFC801CDB7DEB7E8E023
:105630000C94582F6115710589F0DB010D90002045
:10564000E9F7AD0141505109461B570BDC01ED91C3
:10565000FC910280F381E02D0995089580E090E0AF
:105660000895EF92FF920F931F93CF93DF938C01D6
:10567000FB01C0E0D0E064917F018FEFE81AF80AE7
:10568000662361F0D801ED91FC910190F081E02D4D
:10569000C8010995C80FD91FF701EDCFCE01CDB7CD
:1056A000DEB7E6E00C945A2F0E941A2B0895DC0115
:1056B000ED91FC910190F081E02D099508950F93F3
:1056C0001F93CF93DF93EC016DE00E94572B8C0169
:1056D0006AE0CE010E94572B800F911FDF91CF917E
:1056E0001F910F9108950F931F93CF93DF93EC01B8
:1056F0000E94312B8C01CE010E945F2B800F911FE5
:10570000DF91CF911F910F9108950F931F93CF9326
:10571000DF93EC010E941A2B8C01CE010E945F2BBB
:10572000800F911FDF91CF911F910F9108950F93DB
:105730001F93CF93DF93EC010E94572B8C01CE0176
:105740000E945F2B800F911FDF91CF911F910F91CE
:105750000895A1E2B0E0EFEAFBE20C94382F7C015F
:10576000C42EE52FCB01D22E19A221E02D1510F069
:105770002AE0D22E8E010F5D1F4F8D2C912CA12C73
:10578000B12C6C2D7E2FA50194010E94F12E8C2D41
:10579000D29E80191124015011098A3010F4805DC5
:1057A00001C0895CF801808321153105410551054F
:1057B00021F0C22EE32FCA01E4CFB801C7010E9435
:1057C0001A2BA196ECE00C94542FA0E0B0E0EBEE85
:1057D000FBE20C943C2FEC016A017B0121153105A1
:1057E00041F4E881F9810190F081E02D642F099561
:1057F0001DC02A303105A9F477FF12C06DE20E9466
:10580000572B8C0144275527BA014C195D096E09A5
:105810007F092AE0CE010E94A92B800F911F06C0AC
:105820002AE0B701A601CE010E94A92BCDB7DEB7B1
:10583000E8E00C94582F9A01AB01662757FD60955C
:10584000762F0E94E52B08950F931F93CF93DF933C
:10585000EC019A01AB01662757FD6095762F0E94F7
:10586000E52B8C01CE010E945F2B800F911FDF91F1
:10587000CF911F910F9108952115310549F4DC0155
:10588000ED91FC910190F081E02D642F0995089530
:105890000E94A92B08959A01462F50E060E070E025
:1058A0000E943C2C08959A01AB0160E070E00E94D8
:1058B0003C2C08950F931F93CF93DF93EC010E942C
:1058C0003C2C8C01CE010E945F2B800F911FDF9139
:1058D000CF911F910F9108950F931F93CF93DF9353
:1058E000EC019A01AB0160E070E00E943C2C8C015D
:1058F000CE010E945F2B800F911FDF91CF911F91EE
:105900000F9108950F931F93CF93DF93EC019A01AA
:10591000462F50E060E070E00E943C2C8C01CE01EC
:105920000E945F2B800F911FDF91CF911F910F91EC
:105930000895FC0124853585F901E05CFF4F8081E5
:105940009181F901EE5BFF4F20813181821B930B26
:105950008F7399270895FC0184859585FC01E05C8F
:10596000FF4F40815181FC01EE5BFF4F208131816F
:105970004217530741F00190F081E02DE80FF91F25
:10598000808190E008958FEF9FEF0895FC0184855A
:105990009585FC01E05CFF4F40815181FC01EE5B8D
:1059A000FF4F208131814217530779F0A081B181E7
:1059B000A80FB91F8C91208131812F5F3F4F2F732A
:1059C00033273183208390E008958FEF9FEF089570
:1059D000FC0181A1882329F0A489B5898C9186FFD7
:1059E000FBCF11A20895CF93DF93FC012685378565
:1059F000D901A05CBF4F8D919C91119701968F7337
:105A00009927E901CE5BDF4F4881598184179507BB
:105A1000D9F30D90BC91A02DA20FB31F6C93A68556
:105A2000B785A05CBF4F11969C938E93A689B789CA
:105A30002C9181E090E0078C02C0880F991F0A9496
:105A4000E2F7282B2C9381E081A30488F589E02DCF
:105A500080818064808381E090E0DF91CF91089520
:105A600008951F920F920FB60F9211242F933F9318
:105A70004F938F939F93EF93FF938091C00082FD8C
:105A80001CC04091C60080918C0690918D060196B5
:105A90008F73992720918E0630918F068217930776
:105AA00071F0E0918C06F0918D06E45BF94F408334
:105AB00090938D0680938C0602C08091C600FF9162
:105AC000EF919F918F914F913F912F910F900FBE2A
:105AD0000F901F90189586EE95E00E94992C892BC7
:105AE00011F00E94302D08951F920F920FB60F9261
:105AF00011242F933F938F939F93EF93FF932091C4
:105B000048063091490680914A0690914B06281725
:105B1000390731F48091C1008F7D8093C10014C09A
:105B2000E0914A06F0914B06E85FF94F20818091A1
:105B30004A0690914B0601968F73992790934B06D6
:105B400080934A062093C600FF91EF919F918F9119
:105B50003F912F910F900FBE0F901F901895A0E0CE
:105B6000B0E0E5EBFDE20C94382FFC0113821282C9
:105B700088EE93E0A0E0B0E084839583A683B783AA
:105B80008CEB93E091838083758764875787468782
:105B9000318B208B138B028BF58AE48AD78AC68AD5
:105BA000B18EA08E938E828E8F85848F8889858F0B
:105BB0008989868F8A89878F8B8980A3ECE00C94F2
:105BC000542FCF92DF92EF92FF92CF93DF93EC01AD
:105BD0006A017B01411581EE580761057105F9F0F5
:105BE000EC89FD8981E090E008A002C0880F991F30
:105BF0000A94E2F7808360E079E08DE390E0A7010A
:105C000096010E94F12E2150310941095109569502
:105C1000479537952795211580E1380798F0EC894D
:105C2000FD89108260E874E88EE190E0A70196019A
:105C30000E94F12E2150310941095109569547958D
:105C400037952795E889F9893083EA89FB8920838C
:105C500019A2EE89FF89408181E090E09C010C8CC3
:105C600002C0220F331F0A94E2F7422B4083EE89D1
:105C7000FF8940819C010D8C02C0220F331F0A94C2
:105C8000E2F7422B4083EE89FF8940819C010E8C14
:105C900002C0220F331F0A94E2F7422B4083EE89A1
:105CA000FF8920810F8C02C0880F991F0A94E2F7A8
:105CB000809582238083DF91CF91FF90EF90DF90DA
:105CC000CF9008958F929F92AF92BF92CF92DF9222
:105CD000EF92FF920F931F9381E08F9385E08F9354
:105CE00087E08F9383E08F9384E08F93E6EC8E2E92
:105CF000912CF2ECAF2EB12CA1ECCA2ED12CB0EC31
:105D0000EB2EF12C04EC10E025EC30E048E056E0FE
:105D10006CE476E086EE95E00E94AF2D0F900F9038
:105D20000F900F900F901F910F91FF90EF90DF90C9
:105D3000CF90BF90AF909F908F9008950E94E229DE
:105D40000E940F23CBE6DDE20E94BD252097E1F300
:105D50000E946B2DF9CFA29FB001B39FC001A39FFA
:105D6000700D811D1124911DB29F700D811D112494
:105D7000911D08950E94AB2EA59F900DB49F900D8C
:105D8000A49F800D911D11240895B7FF0C94BA2E85
:105D90000E94BA2E821B930B0895DB018F939F9371
:105DA0000E94BA2EBF91AF91A29F800D911DA39F1B
:105DB000900DB29F900D1124089597FB072E16F4B5
:105DC000009407D077FD09D00E946F2F07FC05D003
:105DD0003EF4909581959F4F0895709561957F4F02
:105DE0000895A1E21A2EAA1BBB1BFD010DC0AA1F1C
:105DF000BB1FEE1FFF1FA217B307E407F50720F034
:105E0000A21BB30BE40BF50B661F771F881F991FAE
:105E10001A9469F760957095809590959B01AC01F7
:105E2000BD01CF010895052E97FB1EF400940E943A
:105E30002A2F57FD07D00E94F12E07FC03D04EF405
:105E40000C942A2F50954095309521953F4F4F4FF8
:105E50005F4F089590958095709561957F4F8F4F16
:105E60009F4F08952F923F924F925F926F927F9231
:105E70008F929F92AF92BF92CF92DF92EF92FF925A
:105E80000F931F93CF93DF93CDB7DEB7CA1BDB0B06
:105E90000FB6F894DEBF0FBECDBF09942A883988AB
:105EA00048885F846E847D848C849B84AA84B984B2
:105EB000C884DF80EE80FD800C811B81AA81B981BE
:105EC000CE0FD11D0FB6F894DEBF0FBECDBFED01D2
:105ED0000895EE0FFF1F0590F491E02D0994AA1B81
:105EE000BB1B51E107C0AA1FBB1FA617B70710F0C5
:105EF000A61BB70B881F991F5A95A9F780959095F7
:105F0000BC01CD0108958F929F92AF92BF92CF9224
:105F1000DF92EF92FF92CF93DF93EC01688179815A
:105F20008A819B81611571058105910521F464E2E7
:105F300079ED8BE597E02DE133EF41E050E00E94F1
:105F4000132F49015A019B01AC01A7EAB1E40E9459
:105F5000BA2E6B017C01ACEEB4EFA50194010E9456
:105F6000C82EC60ED71EE81EF91EF7FE06C081E039
:105F7000C81AD108E10880E8F80AC882D982EA8202
:105F8000FB82C701B6019F77DF91CF91FF90EF9021
:105F9000DF90CF90BF90AF909F908F9008950E9418
:105FA000832F089586E091E00E94832F08956093E7
:105FB00006017093070180930801909309010895E9
:105FC0002F923F925F926F927F928F929F92AF92A9
:105FD000BF92CF92DF92EF92FF920F931F93CF93D6
:105FE000DF938B01EA016115710521F0DB018C93D0
:105FF00011969C93209739F09E012250310923324B
:10600000310508F0D8C07C016701BFEFCB1ADB0A6D
:106010005601F7016080862D90E00E941231892B95
:1060200011F07601F1CFFDE26F120AC0570182E054
:10603000A80EB11CD70111966C90772473940BC0F5
:10604000BBE26B1207C05701E2E0AE0EB11CD701F4
:1060500011966C90712CCE018F7E892B89F4B0E360
:106060006B1237C0F50180818F7D8835D1F4618056
:10607000F2E0AF0EB11C872D8260782EC0E1D0E037
:10608000CA30D10551F1C031D10521F0C830D10558
:1060900099F409C0CC24CA94DC2CEC2CAFE0FA2E85
:1060A00022C0209769F7C8E0D0E0CC24CA94DC2C49
:1060B000EC2CFFE1FF2E17C06FEF7FEFCB019E01AD
:1060C000442737FD4095542F0E94F12E69017A0133
:1060D0000AC02097A9F6CAE0D0E0E9E9CE2EDC2C70
:1060E000EC2CE9E1FE2EF50160E020E030E0A901B2
:1060F0004E01AA2497FCA094BA2C1F0170ED572ED4
:10610000560CA9E0A51570F48FEB860D8A3118F4B2
:1061100099EC592E06C08FE9860D8A3148F589EA37
:10612000582E560C852D90E08C179D070CF56F3F6F
:10613000D9F0C216D306E406F50698F0C501B401FD
:106140000E94CD2E9B01AC01852D90E0A0E0B0E037
:10615000280F391F4A1F5B1F281739074A075B079B
:1061600010F46FEF01C061E03196D1016C90C5CFA2
:106170000115110551F0662311F0319703C071FE2E
:1061800004C03297D801ED93FC9370FE07C0509580
:106190004095309521953F4F4F4F5F4F67FF10C09F
:1061A00082E290E090939106809390066FEF7FEFEC
:1061B0008FEF9FEF07C060E070E080E090E002C0EA
:1061C000B901CA01DF91CF911F910F91FF90EF901C
:1061D000DF90CF90BF90AF909F908F907F906F9007
:1061E0005F903F902F900895FC0188279927E894AD
:1061F00021912032E9F3293010F02E30C8F32B32F0
:1062000041F02D3239F4689404C00E944631820F67
:10621000911D219120532A30C0F31EF49095819551
:106220009F4F0895911150C0803219F089508550C8
:10623000D0F7089548EC53E00E941F310895FA0109
:10624000A191B081009719F41097E1F0CD01DC0124
:10625000CD010D90002011F4C00113C0FB0121916C
:10626000222319F02015D9F7F3CFFB012191201536
:1062700019F41E92119606C02223C1F70D9000203A
:10628000A1F7D001FA01A193B08308957AE0979F16
:10629000902D879F802D910D11240895F999FECF9F
:1062A00092BD81BDF89A992780B50895262FF99956
:1062B000FECF1FBA92BD81BD20BD0FB6F894FA9AE9
:1062C000F99A0FBE01960895992788270895F894A2
:0262D000FFCFFE
:1062D20000009206200001000000FF000200020000
:1062E200020002000200020002000200020002009C
:1062F20002000200020002000200028025000005E6
:10630200400AA1204EA50020244EA52C2330C01205
:1063120000001A400AA1204EA5001B1E27522C2362
:10632200308025000005400AA1204EA50020244E01
:10633200A52C2330004B000006400AD0009D4900E6
:106342007B289D492C233000E1000005400A4501CD
:10635200D7DC03B81E0EBF00232E48E801008A4096
:106362000A6001555502AD1E20000023C801545891
:106372002074696D656F75742100596573004E6FE5
:10638200002C00386368004E2F41002C205B005D1A
:106392002028002900486F70206368616E6E656C6A
:1063A200200020402000456E746572696E6720618E
:1063B20064617074697665206368616E6E656C20D5
:1063C20073656C656374696F6E2C207069636B69A9
:1063D2006E673A007363616E6E6572206D6F6465FD
:1063E200004E4F5420454E41424C45440053656E89
:1063F20064696E672073657474696E677320746F65
:106402002052580A00526573657474696E6720736E
:10641200657474696E6773206F6E2052580A00416A
:10642200626F727465642065646974730A00696ED0
:1064320076616C69642073656C656374696F6E0064
:106442000D0A496E76616C696420696E70757420FC
:106452002D2064697363617264656421070053656A
:106462007474696E677320736176656420746F203B
:10647200454550524F4D0A00526576657274656407
:106482002073657474696E67732066726F6D204540
:106492004550524F4D0A004C6F616465642066613D
:1064A20063746F72792064656661756C74730A0037
:1064B2004B657920616E64206368616E6E656C73F2
:1064C2002072616E646F6D697A65640A004F70654F
:1064D2006E4C52536E672054582073746172746903
:1064E2006E672000206F6E20485720006D6F647524
:1064F2006C65206C6F636B65643F00342B3400382D
:1065020000382B340031320031322B340031360066
:1065120050504D0052535349005344410053434C91
:1065220000525844005458440041494E004C4245E0
:1065320045500053504B54524D0053425553005353
:10654200554D44004C4C494E440000070B0C1011B1
:106552001500B7012B032F033103350338033D0325
:10656200B7014003440349034D0351035503590343
:106572005D0363036A036F0374038D028D028D0250
:106582008D02160A1322312900000000F32CF82A8A
:08659200992CC62CAB2CE82C5F
:107E00000F92CDB7DEB7112484B714BE81FFF1D035
:107E100082E08093C00088E18093C10086E0809377
:107E2000C20080E18093C4008EE0CDD088249924E4
:107E3000CC24C394F5E0DF2EE1E1EE2E73E0F72EC3
:107E4000B6D0082F813479F4B2D08983C2D0898129
:107E5000823811F481E005C0813811F485E001C059
:107E600083E09ED09AC0823411F484E103C085344B
:107E700019F485E0B6D091C0853561F498D0082F0B
:107E800010E095D090E0982E8824802A912A880CC2
:107E9000991C82C0863521F484E0A3D080E0E1CF34
:107EA000843609F04CC083D082D0A82E80D0B82E62
:107EB00000E011E07CD0F80181938F01AE16D1F77C
:107EC00088D0FB2DF53489F4E0E0F1E00BC0F9999E
:107ED000FECF92BC81BC0894811C911C819180BD15
:107EE000FA9AF99AEA1598F358C08B2D863409F05E
:107EF00054C0F401F7BEE89507B600FCFDCFF401CD
:107F0000A0E0B1E02C9130E011968C91119790E0B7
:107F1000982F8827822B932B12960C01C7BEE895C9
:107F20001124329681E0A038B80761F7F401D7BE7A
:107F3000E89507B600FCFDCFE7BEE8952EC0843774
:107F4000F1F435D034D0182F32D0B82E42D0FB2DDA
:107F5000F63421F4F40105914F010CC0FB2DF534EA
:107F600049F4F999FECF92BC81BC0894811C911C04
:107F7000F89A00B5802F14D0115049F70EC08537FC
:107F800039F427D08EE10CD085E90AD08FE069CF93
:107F9000813511F488E017D01CD080E101D050CF9A
:107FA0009091C00095FFFCCF8093C600089580910A
:107FB000C00087FFFCCF8091C00084FD01C0A89560
:107FC0008091C6000895E0E6F0E098E19083808318
:107FD0000895EDDF803219F088E0F5DFFFCF84E10E
:107FE000DFCF1F93182FE3DF1150E9F7F2DF1F9166
:0E7FF0000895282E80E0E7DFEE27FF27099492
:027FFE0001057B
:0400000300007E007B
:00000001FF
